S0220000687474703A2F2F737265636F72642E736F75726365666F7267652E6E65742F1D
S3250800280000000120CDAD0008094B00080B4B00080D4B00080F4B0008114B00080000000027
S32508002820000000000000000000000000A18B0008134B000800000000418C0008154B0008B3
S325080028401DAE00081DAE00081DAE00081DAE00081DAE00081DAE00081DAE00081DAE0008D2
S325080028601DAE00081DAE00081DAE00081DAE00082D4B00083D4B00081DAE00081DAE000848
S325080028801DAE00081DAE00084D4B00085D4B00086D4B00087D4B00088D4B00081DAE0008F1
S325080028A01DAE00081DAE00081DAE00081DAE00081DAE000800000000000000001DAE000818
S325080028C01DAE000800000000000000009D4B0008000000001DAE00081DAE00080000000081
S325080028E01DAE00081DAE000800000000000000000000000000000000000000000000000024
S325080029000000000000000000000000001DAE000800000000000000001DAE00081DAE000830
S325080029201DAE00081DAE0008AD4B00081DAE00081DAE00080000000000000000000000003D
S325080029401DAE00081DAE00081DAE00081DAE00081DAE00081DAE00081DAE00081DAE0008D1
S325080029601DAE00081DAE00081DAE0008000000001DAE00081DAE000800000000000000002A
S325080029801DAE00081DAE00081DAE0008EE11AA5581F0004102E000BF83F0004330B54FEA8B
S325080029A041044FEA430594EA050F08BF90EA020F1FBF54EA000C55EA020C7FEA645C7FEA58
S325080029C0655C00F0E2804FEA5454D4EB5555B8BF6D420CDD2C4480EA020281EA030382EAC2
S325080029E0000083EA010180EA020281EA0303362D88BF30BD11F0004F4FEA01314FF4801C4A
S32508002A004CEA113102D0404261EB410113F0004F4FEA03334CEA133302D0524263EB430317
S32508002A2094EA050F00F0A780A4F10104D5F1200E0DDB02FA0EFC22FA05F2801841F1000185
S32508002A4003FA0EF2801843FA05F359410EE0A5F120050EF1200E012A03FA0EFC28BF4CF0D9
S32508002A60020C43FA05F3C01851EBE37101F0004507D54FF0000EDCF1000C7EEB00006EEBA3
S32508002A800101B1F5801F1BD3B1F5001F0CD349085FEA30004FEA3C0C04F101044FEA44523B
S32508002AA012F5800F80F09A80BCF1004F08BF5FEA500C50F1000041EB045141EA050130BDA0
S32508002AC05FEA4C0C404141EB0101013C28BFB1F5801FE9D291F0000F04BF01460020B1FA0F
S32508002AE081F308BF2033A3F10B03B3F120020CDA0C3208DD02F1140CC2F10C0201FA0CF0FE
S32508002B0021FA02F10CE002F11402D8BFC2F1200C01FA02F120FA0CFCDCBF41EA0C0190407B
S32508002B20E41AA2BF01EB0451294330BD6FEA04041F3C1CDA0C340EDC04F11404C4F12002CE
S32508002B4020FA04F001FA02F340EA030021FA04F345EA030130BDC4F10C04C4F1200220FA54
S32508002B6002F001FA04F340EA0300294630BD21FA04F0294630BD94F0000F83F4801306BF0D
S32508002B8081F480110134013D4EE77FEA645C18BF7FEA655C29D094EA050F08BF90EA020F72
S32508002BA005D054EA000C04BF1946104630BD91EA030F1EBF0021002030BD5FEA545C05D11C
S32508002BC04000494128BF41F0004130BD14F580043CBF01F5801130BD01F0004545F0FE4131
S32508002BE041F470014FF0000030BD7FEA645C1ABF194610467FEA655C1CBF0B46024650EA66
S32508002C00013406BF52EA033591EA030F41F4002130BD00BF90F0000F04BF0021704730B59A
S32508002C204FF4806404F132044FF000054FF0000150E700BF90F0000F04BF0021704730B5AB
S32508002C404FF4806404F1320410F0004548BF40424FF000013EE700BF42004FEAE2014FEA8B
S32508002C6031014FEA02701FBF12F07F4393F07F4F81F06051704732F07F4208BF704793F0B9
S32508002C807F4F04BF41F40021704730B54FF4607401F0004521F000411CE700BF50EA010205
S32508002CA008BF704730B54FF000050AE050EA010208BF704730B511F0004502D5404261EBEA
S32508002CC041014FF4806404F132045FEA915C3FF4D8AE4FF003025FEADC0C18BF03325FEA99
S32508002CE0DC0C18BF033202EBDC02C2F1200300FA03FC20FA02F001FA03FE40EA0E0021FADD
S32508002D0002F11444BDE600BF70B54FF0FF0C4CF4E06C1CEA11541DBF1CEA135594EA0C0FAF
S32508002D2095EA0C0F00F0DEF82C4481EA030621EA4C5123EA4C5350EA013518BF52EA033532
S32508002D4041F4801143F4801338D0A0FB02CE4FF00005E1FB02E506F00042E0FB03E54FF021
S32508002D600006E1FB03569CF0000F18BF4EF0010EA4F1FF04B6F5007F64F5407404D25FEA5D
S32508002D804E0E6D4146EB060642EAC62141EA55514FEAC52040EA5E504FEACE2EB4F1FD0C21
S32508002DA088BFBCF5E06F1ED8BEF1004F08BF5FEA500E50F1000041EB045170BD06F0004631
S32508002DC046EA010140EA020081EA0301B4EB5C04C2BFD4EB0C0541EA045170BD41F4801155
S32508002DE04FF0000E013C00F3AB8014F1360FDEBF002001F0004170BDC4F10004203C35DA93
S32508002E000C341BDC04F11404C4F1200500FA05F320FA04F001FA05F240EA020001F0004235
S32508002E2021F0004110EBD37021FA04F642EB06015EEA430E08BF20EAD37070BDC4F10C040C
S32508002E40C4F1200500FA04F320FA05F001FA04F240EA020001F0004110EBD37041F10001CA
S32508002E605EEA430E08BF20EAD37070BDC4F1200500FA05F24EEA020E20FA04F301FA05F254
S32508002E8043EA020321FA04F001F0004121FA04F220EA020000EBD3705EEA430E08BF20EAFC
S32508002EA0D37070BD94F0000F0FD101F00046400041EB010111F4801F08BF013CF7D041EAE2
S32508002EC0060195F0000F18BF704703F00046520043EB030313F4801F08BF013DF7D043EA5D
S32508002EE00603704794EA0C0F0CEA135518BF95EA0C0F0CD050EA410618BF52EA4306D1D141
S32508002F0081EA030101F000414FF0000070BD50EA410606BF1046194652EA430619D094EAAF
S32508002F200C0F02D150EA013613D195EA0C0F05D152EA03361CBF104619460AD181EA030181
S32508002F4001F0004141F0FE4141F470014FF0000070BD41F0FE4141F4780170BD70B54FF000
S32508002F60FF0C4CF4E06C1CEA11541DBF1CEA135594EA0C0F95EA0C0F00F0A7F8A4EB05049D
S32508002F8081EA030E52EA03354FEA013100F088804FEA03334FF0805545EA131343EA126356
S32508002FA04FEA022245EA111545EA10654FEA00260EF000419D4208BF964244F1FD0404F562
S32508002FC0407402D25B084FEA3202B61A65EB03055B084FEA32024FF480104FF4002CB6EBB0
S32508002FE0020E75EB030E22BFB61A754640EA0C005B084FEA3202B6EB020E75EB030E22BFCD
S32508003000B61A754640EA5C005B084FEA3202B6EB020E75EB030E22BFB61A754640EA9C006D
S325080030205B084FEA3202B6EB020E75EB030E22BFB61A754640EADC0055EA060E18D04FEAAA
S32508003040051545EA16754FEA06164FEAC30343EA52734FEAC2025FEA1C1CC0D111F4801F95
S325080030600BD141EA00014FF000004FF0004CB6E711F4801F04BF01430020B4F1FD0C88BF13
S32508003080BCF5E06F3FF6AFAEB5EB030C04BFB6EB020C5FEA500C50F1000041EB045170BDDB
S325080030A00EF0004E4EEA113114EB5C04C2BFD4EB0C0541EA045170BD41F480114FF0000ECC
S325080030C0013C90E645EA060E8DE60CEA135594EA0C0F08BF95EA0C0F3FF43BAF94EA0C0F6B
S325080030E00AD150EA01347FF434AF95EA0C0F7FF425AF104619462CE795EA0C0F06D152EACC
S3250800310003353FF4FDAE1046194622E750EA410618BF52EA43067FF4C5AE50EA41047FF418
S325080031200DAF52EA43057FF4EBAE12E74FEA4102B2F1E04324BFB3F5001CDCF1FE5C0DD946
S3250800314001F0004C4FEAC0024CEA5070B2F1004F40EB830008BF20F00100704711F0804F34
S3250800316021D113F13872BCBF01F00040704741F480114FEA5252C2F11802C2F1200C10FAE5
S325080031800CF320FA02F018BF40F001004FEAC1234FEAD32303FA0CFC40EA0C0023FA02F375
S325080031A04FEA4303CCE77FEA625307D150EA01331EBF4FF0FE4040F44000704701F00040B5
S325080031C040F0FE4040F40000704700BF10B5054C237833B9044B13B10448AFF30080012387
S325080031E0237010BD0001002000000000F4AF000808B5034B1BB103490348AFF3008008BD40
S325080032000000000004010020F4AF000808B500F0A3FB00F0010400F091FE044000F058FD88
S32508003220044000F0A5FD044000F030FF044000F0F3FB044001F02AF8044000F0C5FD044094
S3250800324000F0C6F9044000F00DF904421AD104F083FF022000F0FCFE0D4B1B689B0B6422BD
S3250800326002FB03F3002BF4D000BF00BF00BF00BF00BF00BF00BF00BF00BF00BF00BF00BF6A
S32508003280013BEFE7034B186804F0DAFFFEE700BF9C0000201C01002008B5054A002105485C
S325080032A004F06FFF044B1860003818BF012008BD1CB000080D3200081C01002000B585B0A0
S325080032C0EC468CE80F0000231A4661460548006805F0D2F90121044B186805F05FF805B09A
S325080032E05DF804FB200100202401002008B50146024B186805F052F808BD00BF240100200D
S3250800330030B589B04FF0FF33002207215248006805F091F8044610F0010F0AD114F0020FFC
S3250800332040F0968014F0040FECD0002000F00AF9E8E700231A4602A94848006805F0DEF992
S325080033409DF808509DF81130012B1DD0022B3BD0002BE3D1072D43D86AB2002ADED0013DEB
S32508003360062DDBD801A252F825F000BFF1330008F9330008013400081D3300080F34000858
S325080033801934000831340008132D08D9FF228DF81820059A012106A800F05EFDBEE7284691
S325080033A000F0A6FA01908DF8185004220DF119010DEB020001F024FC9DF81130059A05210D
S325080033C006A800F049FDA9E704220DEB02010DF1090001F015FC0199284600F035FA9DE796
S325080033E0FF2D9BD1002000F0ADF802F095FE95E7012000F0A7F891E7002000F0A3F88DE72A
S3250800340040F6B831164B186804F08CFF86E70021132000F05FFA81E706228DF818200122A5
S325080034208DF81920059A022106A800F015FD75E704220DEB02010DF1090001F0E1FB9DED73
S32508003440010A00F073FC9DED010A00F0AFFC65E7022000F0FDFD65E724010020200100209A
S325080034603001002070B5254804F076FF244B1860041E18BF0124234A0021234804F081FE81
S32508003480224B186000280CBF002404F00104204A1021082005F0A5F81E4B186000280CBF00
S325080034A0002404F001041C4E1C4B02220121304604F0E4FE1A4D286000280CBF002404F084
S325080034C00104184B02220121304604F0D7FE164B186000280CBF002404F001044FF47A71DA
S325080034E0286804F01FFF002814BF002404F001040E4800F0D9FC204670BD00BFB0B000082F
S3250800350024010020C0B00008013300082801002098B0000820010020ED320008E4B0000807
S325080035202C010020F4B0000830010020BD32000808B50146024B186804F030FF08BD00BFC4
S325080035403401002010B504460146032000F044FD2146122000F0BEF910BD08B5122000F072
S32508003560DBF908BD0000000008B5F2EE087AB4EEE70AF1EE10FA01DDB0EE670AF8EE087AB4
S32508003580B4EEE70AF1EE10FA01D5B0EE670A10EE100AFFF761FB0AA3D3E90023FFF7FEF9D9
S325080035A009A3D3E90023FFF7D9FCFFF7BFFD00EE100A00F0FBFB00F0010008BDAFF300802F
S325080035C04A0C022B8716344077BE9F1A2F0D414038B5174A0021174804F0D3FD164B186033
S325080035E0041E18BF0124154804F0B6FE144B186000280CBF002404F00104124B01221146DC
S32508003600114804F03BFE114D286000280CBF002404F001049FED0E0AFFF7A6FF64212868CC
S3250800362004F080FE002814BF002004F0010038BD48B10008553600083801002038B1000827
S32508003640340100206CB10008313500083C0100200000000008B52DED088BDFED438AB0EE76
S32508003660688A05E0DFED408AB0EE6A0AFFF77CFFF0EE689AB0EE489A4FF0FF330022012137
S325080036803A48006804F0D7FE10F0010FF4D0384803F027FAFFF761FF9FED338AF0EE488AB2
S325080036A00028E5D0002000F037F9002848D1022000F036F9F0EE408A032000F031F9B0EEDA
S325080036C040AA042000F02CF9B0EE40BA062000F027F9F0EE40AA072000F022F9F0EE40BA19
S325080036E0092000F01DF9B0EE408A052000F018F938EE408A68EE887ADFED1E6A68EE268A5D
S3250800370078EEA98A2AEE28AA38EE497A27EE0B7A87EE266A77EE8A7A77EE867AF4EEE7AA4F
S32508003720F1EE10FA9ED4F4EEE7BAF1EE10FA02DCF0EE67AA98E7F0EE6BAADFED0B8A93E79A
S32508003740002000F0E9F8012804D0F0EE698AB0EE498A8DE700F0E4F8FFF706FFDFED028A98
S32508003760B0EE688A84E700BF0000000034010020F4030020CDCCCC3D01288CBF00200120BE
S3250800378070470000084B03EB00139B688B4207D8054B03EB0013DB688B4203D20020704754
S325080037A0002070470120704788B10008084B03EB00139B688B4207DC054B03EB0013DB6870
S325080037C08B4203DA00207047002070470120704788B100080C4B03EB0013D3ED027AF4EEF4
S325080037E0C07AF1EE10FA0BD8074B03EB0013D3ED037AF4EEC07AF1EE10FA03DA002070476C
S32508003800002070470120704788B1000808B503010C4AD35C13F0010F09D113F0020F0BD187
S3250800382013F0040F0BD00846FFF7A6FF03E000EE101AFFF7CFFF08BDFFF7B8FFFBE7FFF797
S32508003840A1FFF8E788B1000838B503010D4AD35C13F0080F00D038BD04460D464FF0FF3138
S32508003860094B186804F06BFE29462046FFF7CEFF10B1064B43F83450034B186804F08BFE55
S32508003880E9E700BF88B10008E00100204001002038B504460D464FF0FF310C4B186804F024
S325080038A04EFE29462046FFF7B1FF30B9084B03EBC4031A7942F002021A71054B43F83450DF
S325080038C0024B186804F067FE38BD00BFE00100204001002008B5FFF7DBFF08BD00B583B064
S325080038E08DED010A0199FFF7D3FF03B05DF804FB38B50446064D4FF0FF31286804F01FFE32
S32508003900044B53F83440286804F045FE204638BDE00100204001002008B5FFF7E9FF08BDA7
S3250800392008B5FFF7E5FF00EE100A08BD08B5034B03EB00135968FFF7ABFF08BD88B10008A2
S3250800394010B5002404E0E0B2FFF7F0FF0134A4B2132CF8D910BD000010B5064804F0A5FD04
S32508003960054B1860041E18BF0124FFF7E9FF204610BD00BFC8B20008E001002008B572B120
S325080039800D4B60F07F00187000225A7099700B480323838100F088FB00F0010008BD064B7E
S325080039A060F07F001870597004480223838100F07BFB00F00100F1E7EC0100200000002008
S325080039C010B50C4692B1114B187000225A709A700F480323838100F067FB00F001000D4B89
S325080039E05A789B7843EA0223238010BD074B187000225A7006480223838100F055FB00F0A5
S32508003A000100044B5B782380EFE700BFEC01002000000020E401002038B5144804F045FD8C
S32508003A20134D2860041E18BF01244FF0FF3104F086FD002000F062FA002282211046FFF70F
S32508003A409DFF0440002000F069FA012000F056FA002282211046FFF791FF0440012000F0AE
S32508003A605DFA286804F097FD204638BDE4B20008F40100202DE9F04182B00F4690460023F4
S32508003A800B70ADF8063018B1012854D0012600E001263F4D4FF0FF31286804F050FD30463C
S32508003AA000F02CFA0022A0211046FFF767FF00F00104304600F032FA286804F06CFD642055
S32508003AC004F0CDFB4FF0FF31286804F038FD304600F014FA01220DF106011046FFF770FF9D
S32508003AE00440304600F01AFA286804F054FD24B3BDF8063013F0010F24D15B08ADF806301D
S32508003B00A8F80030224D4FF0FF31286804F017FD304600F0F3F9002284211046FFF72EFFBF
S32508003B200440304600F0FAF9286804F034FD204602B0BDE8F0810026ABE73B7843F0020354
S32508003B403B70F4E7124C4FF0FF31206804F0F7FC304600F0D3F9002239460720FFF730FF76
S32508003B60304600F0DBF9304600F0C8F9002282211046FFF703FF304600F0D0F9206804F018
S32508003B800AFD3B7843F001033B700024CFE700BFF401002010B52DED028B88B0012004F014
S32508003BA05EFB08224149424801F0B0FD6EE004244FF0FF313F4B186804F0C1FC00230AE015
S32508003BC0E1183A4A32F8111008AA02EB830242F8101C01339BB2032BF2D9002325E008AA31
S32508003BE002EB830151ED047AF8EE677A9FED327A67EE877A9FED317A67EE877A304A92EDAF
S32508003C00007A67EE877A2F4A02EB830292ED007A67EE277A2C4A02EB830292ED007A77EEA6
S32508003C20C77A41ED087A01339BB2032BD7D9DDED028AB0EE680A0B20FFF750FE9DED038A3A
S32508003C40B0EE480A0C20FFF749FE88EE880A0D20FFF744FE28EE880A0D20FFF73FFEDDEDBE
S32508003C60008AB0EE680A0F20FFF738FE9DED018AB0EE480A1020FFF731FE28EE880A11200E
S32508003C80FFF72CFE0B4B186804F085FC4FF0FF33002203210D48006804F0CDFB10F0020F6A
S32508003CA085D110F0010FF1D0002481E7F8010020280200200C0200200000803D000080393C
S32508003CC04400002020B3000830B300080802002010B50F4A00210F4804F053FA0E4B1860DA
S32508003CE0041E18BF01240D4804F036FB0C4B186000280CBF002404F001040A4804F0D5FB29
S32508003D00094B186000280CBF002004F0010010BD60B30008953B00081002002050B30008C4
S32508003D200802002040B300080C020020014B83ED000A70474400002008B50221024B186894
S32508003D4004F02CFB08BD00BF0802002008B50121024B186804F022FB08BD00BF0802002021
S32508003D60836D836D836D836DC36CDB6B7047000008B50021034802F007FAB0FA80F04009CA
S32508003D8008BD00BFB4020020DFED067A20EE270A054B93ED007AC0EE077AFCEEE77A17EE67
S32508003DA0900A704700F07F454800002008B5FFF7EBFF034600221146024802F017FA00F0EC
S32508003DC0010008BDB402002070B5042000F020F91D4C237803432370032000F019F923784A
S32508003DE043EA40032370022000F012F9237843EA80032370012000F00BF9237843EAC0001A
S32508003E00C0B22070114E336843EA40133360104D1049284601F01BFE04463146284601F037
S32508003E2016FE0443E4B2284601F094FE0443E4B20221284601F0D6FF204310F0FF0F0CBF22
S32508003E400120002070BD00BF180200204C0000208C02002074000020082901D9002070475D
S32508003E6000B587B012021FFA82FC4CEA03130C4A1278134343F41073009300230193029382
S32508003E80039304918DF81430012302466946054801F08EFEB0FA80F0400907B05DF804FBCD
S32508003EA0180200208C020020014B1860704700BF1402002030B58FB005AB07AA002101F005
S32508003EC0ECFE079BC3F300220492C3F301138DF80D309DF82C208DF80C2001AC214605A8FB
S32508003EE000F08EFE034B1D6894E80F00A8470FB030BD00BF14020020436A704708B5064BD8
S32508003F004FEA401C03EB4010027F818853F80C0002F0EDFC08BD00BF24B4000808B5064B92
S32508003F204FEA401C03EB4010027E818853F80C0002F0DDFC08BD00BF24B4000870B582B03A
S32508003F40224B1A6E42F001021A661B6E03F001030193019B012500240BE000231D401C4BDD
S32508003F604A0103EB41110431985802F0E1FB0134E4B2042C08D82146154B03EB44139B68CB
S32508003F80002BEAD10123E9E700240EE001231D402046FFF7C3FF0F4B720103EB4611043141
S32508003FA0985802F0C5FB0134E4B2032C0AD82646084B03EB44139B68012BE8D0112BE5D099
S32508003FC00023E4E7284602B070BD00BF0010024084B3000824B4000808B559B10B4B4FEA12
S32508003FE0401C03EB4010027F818853F80C0002F07EFC08BD054B4FEA401C03EB4010027E64
S32508004000818853F80C0002F072FCF2E724B4000838B504460D4B420103EB4015A9889858E3
S3250800402002F05EFCEB69012B07D0084B03EB44139B69012B05D0002038BD0128F5D101200D
S32508004040FAE708B10020F7E70120F5E784B3000808B5044B420103EB40108188985802F006
S325080040604BFC08BD24B400080246002008B10020704700EB8003044951F823309342F7D05B
S32508004080431CD8B2F2E700BFC8B4000808B5044804F062F9034B1860003818BF012008BDFA
S325080040A0ECB400081C02002038B504460378244D03EB830305EB83034FF0FF31586804F0DC
S325080040C03EFA237803EB830305EB8303D96841F002011C4B186804F08EF9237803EB830032
S325080040E0A389A268616855F8200003F0DBFD00280CBF0125002511D00020237810F0020F90
S3250800410005F0010518BF002503EB83030C4A02EB8303586804F03FFA284638BD237803EB84
S325080041208303074A02EB8303D9684FF0FF33002241F002010348006804F07DF9DDE700BF7F
S32508004140C8B400081C02002008B5FFF78DFF00EB8000044B03EB8003D968034B186804F022
S325080041601DF908BDC8B400081C02002008B5FFF77BFF00EB8000044B03EB8003D968034BAD
S32508004180186804F00BF908BDC8B400081C02002008B5026E826DD26B436DDB6BFFF764FF6A
S325080041A00221024B186804F0F9F808BD1C02002000EE100AB8EEC00ADFED097A20EE270A13
S325080041C0DFED087A60EE277A9FED077A77EE877A20EE270ADFED057A30EE670A704700BF92
S325080041E000000039DB8A1F416DE76B4342E0754310B52DED028B84B000238DF80F300A2026
S3250800420004F02DF8012422E01F4B019300238DF80F30012429E0BDF80C00FFF7C9FF8DED44
S32508004220020ADDED018AB0EE680A0820FFF756FB9DED028AB0EE480A0920FFF74FFB38EEFB
S32508004240C80A0A20FFF74AFB642004F008F803AA0DF10F010020FFF70DFC0440D4D0BDF82A
S325080042600C00FFF7A5FF8DED010A03AA0DF10F010120FFF7FFFB0440CDD1034B0293002351
S325080042808DF80F300124CCE77B9488C308B5054A0021054803F075FF044B1860003818BF63
S325080042A0012008BD08B50008F141000820020020014A024B9A6070470028000800ED00E083
S325080042C02DE9F04188B0002403940494059406940794364BDA6C42F00402DA64DA6C02F0BB
S325080042E004020092009ADA6C42F00102DA64DA6C02F001020192019ADA6C42F00202DA64A2
S32508004300DB6C03F002030293029B294F22464FF48041384602F0EBFA22464FF480714FF00A
S32508004320904002F0E4FA234D22466021284602F0DEFA4FF4804303930126049605940694AE
S3250800434003A9384602F0F4F94FF40048CDF80C800494059403A9384602F0EAF94FF4807304
S32508004360039304960594069403A94FF0904002F0DFF9CDF80C800494059403A94FF090400A
S3250800438002F0D6F9982303930494059403A9284602F0CEF96023039304960594069403A967
S325080043A0284602F0C5F908B0BDE8F08100100240000800480004004800B583B0164B9A6CC6
S325080043C042F001029A649A6C02F001020092009A9A6C42F002029A649B6C03F002030193A8
S325080043E0019B002205210C2001F050FE0C2001F085FE002205210D2001F048FE0D2001F0F6
S325080044007DFE002205213A2001F040FE3A2001F075FE03B05DF804FB0010024008B5FEF779
S325080044203BFF024B186803F00BFFFEE72402002072B6FEE700B587B0002300930193029367
S325080044400393049305932F482F4A026043608360C3600122026108214161037642760421E7
S32508004460C16180F820308362C36280F83020436380F838201C21C163802101644364826408
S3250800448000F024FC002832D1204B009306230193072302937F2303930423049300230593A8
S325080044A06946184800F072FE18BB194B00930C2301936946134800F069FEE0B9154B009305
S325080044C01223019369460F4800F060FEA8B9124B00931823019369460A4800F057FE70B922
S325080044E07F21084801F0BCF907B05DF804FBFFF79FFFFFF79DFFFFF79BFFFFF799FFFFF7D3
S3250800450097FF00BF280200200000045040002019000021438000501D0080F03E08B50D4810
S325080045200D4B03602023436000238360C3604FF4402202614FF4A0024261037643768376E8
S325080045400122C2760377437701F0DBF900B908BDFFF76EFF8C0200200064004000B58BB0D6
S325080045602422002101A806F05AFC1048104B036001F0F8FD98B90022019202920392049210
S32508004580059201A9094801F048FE50B9002201A9064801F0DDFE30B90BB05DF804FBFFF767
S325080045A047FFFFF745FFFFF743FF00BFB40200200074004008B51048104B03604FF48273E1
S325080045C04360002383604FF4E062C2600361012242614FF4007282613022C261036243623C
S325080045E083620722C2620363436303F0EBFA00B908BDFFF71DFF00BF0404002000300140AF
S3250800460008B51148114B0360114B4360002383600122C260036143618361C361036202F006
S3250800462074F950B90021084802F0CDF938B90021054802F0F6F920B908BDFFF7F9FEFFF70C
S32508004640F7FEFFF7F5FE00BFA003002000540040EC9C901008B50848084B036006234360A1
S3250800466040F6FF73C3609623836002F006FA00B908BDFFF7DDFE00BFF4030020003000403E
S3250800468000B597B04422002105A806F0C8FB0023009301930293039304934FF4007002F072
S325080046A02FFA30BB092305934FF4A023069301230A9302230F93032210920422119210222B
S325080046C01292072213921493159305A802F002FB88B90F2300930323019300230293039361
S325080046E004930421684602F02BFE30B917B05DF804FBFFF79DFEFFF79BFEFFF799FE000076
S3250800470008B5FFF7D5FD00F0ABFAFFF7B9FFFFF7D7FDFFF751FEFFF78DFEFFF7FFFEFFF74A
S325080047201DFFFFF747FFFFF76BFFFFF793FF03F0E5FC054A0021054803F023FD044B1860C0
S3250800474003F0EEFCFEE700BF34B500081D4400082402002000B583B00D4B1A6E42F001022D
S325080047601A661A6E02F001020092009A9A6D42F080529A659B6D03F080530193019B0022D8
S325080047800F216FF0010001F081FC03B05DF804FB0010024070B59EB00446002119911A9181
S325080047A01B911C911D91542204A806F038FB2268334B9A4201D01EB070BD4FF4804304934C
S325080047C04FF04053169304A802F034FF002850D12C4BDA6C42F40052DA64DA6C02F4005225
S325080047E00192019ADA6C42F00102DA64DA6C02F001020292029ADA6C42F00202DA64DB6C58
S3250800480003F002030393039B062319930B261A9600251B9519A94FF0904001F089FF032363
S3250800482019931A961B9519A9174801F081FF1748174B036045608560C560802303614FF4AF
S32508004840807343614FF4806383612023C3614FF40053036201F022FE70B90C4BE3649C6271
S3250800486000220521122001F011FC122001F046FCA1E7FFF7DDFDABE7FFF7DAFDEDE700BF03
S32508004880000004500010024000040048C80200203004024000B589B00023039304930593E2
S325080048A0069307930268244B9A4202D009B05DF804FB03F5D6339A6D42F000729A659A6D71
S325080048C002F000720192019ADA6C42F00102DA64DB6C03F001030293029B4FF4C053039323
S325080048E002230493032306930923079303A94FF0904001F01DFF00220521132001F0C6FB74
S32508004900132001F0FBFB00220521142001F0BEFB142001F0F3FB00220521152001F0B6FB17
S32508004920152001F0EBFB00220521162001F0AEFB162001F0E3FBB9E70064004000B589B00E
S325080049400023039304930593069307930268124B9A4202D009B05DF804FB03F5CE339A6DAC
S3250800496042F000529A659A6D02F000520192019ADA6C42F00102DA64DB6C03F001030293A1
S32508004980029B102303930323049303A94FF0904001F0CEFEDEE700BF0074004010B59CB025
S325080049A0044600211791189119911A911B91542202A806F034FA2268184B9A4201D01CB082
S325080049C010BD4023029302A802F034FE18BB144CE36C43F00103E364E36C03F0010300935D
S325080049E0009B4FF4C0631793122318930023199303231A9304231B9317A94FF0904001F0E7
S32508004A0097FEA36D43F40013A365A36D03F400130193019BD3E7FFF70BFDD8E7005400403C
S32508004A200010024010B588B000230393049305930693079302682F4B9A4201D008B010BDE8
S32508004A40044603F560431A6E42F480521A661A6E02F480520192019ADA6C42F00102DA641C
S32508004A60DB6C03F001030293029BE023039302230493032306930523079303A94FF0904027
S32508004A8001F056FE1C481D4B03600123436000238360C3608022026143618361C36103628E
S32508004AA001F0FCFC00BB144BA3659C621448154B036001234360102383600023C3608022FB
S32508004AC0026143618361C361036201F0E7FC70B90B4B63659C6200220521232001F0D6FAEF
S32508004AE0232001F00BFBA9E7FFF7A2FCDBE7FFF79FFCEDE700300140100300201C00024021
S32508004B005803002030000240FEE7FEE7FEE7FEE7FEE7704708B500F0B3F805F08DFD01286A
S32508004B2000D108BD04F0BEF8FBE7000008B5024801F09BFD08BD00BF1003002008B50248F7
S32508004B4001F093FD08BD00BF5803002008B5024800F0B0F908BD00BF2802002008B5024852
S32508004B6001F05DF908BD00BF8C02002008B5024801F055F908BD00BF8C02002008B502482F
S32508004B8001F04DF908BD00BF8C02002008B5024801F045F908BD00BF8C02002008B502482F
S32508004BA003F00EFA08BD00BF0404002008B5024801F05BFD08BD00BFC80200200E4AD2F860
S32508004BC0883043F47003C2F888300C4B1A6842F001021A60002199601A6822F0A85222F4AD
S32508004BE010221A604FF48052DA601A6822F480221A609961704700BF00ED00E00010024069
S32508004C0008B50B460146184606F08EF908BD0000104B1B780BB90120704710B504464FF4B5
S32508004C207A70B0FBF3F30C4A1068B0FBF3F001F085FA68B90F2C01D901200AE00022214655
S32508004C404FF0FF3001F022FA044B1C60002000E0012010BDA00000209C000020A4000020D2
S32508004C6010B5032001F000FA0F20FFF7D1FF10B10124204610BD0446FFF76CFDF9E70000BC
S32508004C80034B1B78034A11680B441360704700BFA000002068040020014B1868704700BF99
S32508004CA06804002038B50446FFF7F6FF0546B4F1FF3F02D0044B1B781C44FFF7EDFF401BB9
S32508004CC0A042FAD338BD00BFA000002030B583B000230193002800F0DA800446436D13B3A2
S32508004CE023689A6812F0005F05D09A6822F0204222F03F029A602268936813F0805F1FD1C9
S32508004D00936823F0104323F03F0343F080539360604B1B689B09604AA2FB03239B090133BF
S32508004D205B00019309E0FFF735FD0023A36584F85030D5E7019B013B0193019B002BF9D185
S32508004D402268936813F0805F78D1636D43F010036365A36D43F00103A3650120936813F049
S32508004D60040300D00123616D11F0100F40F08880002B40F08580636D23F4817343F0020391
S32508004D806365936813F0010F0BD1444B9B6813F0010F06D1636842498A6822F47C12134395
S32508004DA08B60627E636B43EA4233E2681343A268134394F8202043EA0243012A40D0A26A25
S32508004DC022B102F47072E16A0A4313432168CD68344A2A401A43CA6021688B6813F0040379
S32508004DE000D001238A6812F0080200D00122B3B9AAB9237E94F83020520042EA8332CB680E
S32508004E0023F4804323F002031343CB6094F83830012B1AD02268136923F0010313612369EA
S32508004E20012B24D02268136B23F00F031363636D23F0030343F00103636526E000208DE71F
S32508004E40626A013A43EA4243B9E721680B6923F4FF6323F00403E26B256C2A43656C2A43D2
S32508004E60A56C2A43134343F001030B61D7E721680B6B23F00F03E269013A13430B63D6E7C4
S32508004E80636D43F010036365012003B030BD0120FBE700BF9C000020632D3E0500000450C0
S32508004EA00003045007C0F0FF08B5806AFEF74EFF08BD704770B5044603681E685D6816F047
S32508004EC0020F10D015F0020F0DD0436D13F0100F03D1436D43F400634365204600F010FDE5
S32508004EE0236802221A6016F0040F02D015F0040F05D116F0080F3AD015F0080F37D0636D88
S32508004F0013F0100F03D1636D43F4007363652368DA6812F4406F24D1DA6812F4005F20D13C
S32508004F201A6812F0080F1CD09A6812F0040F10D15A6822F00C025A60636D23F480736365A6
S32508004F40636D13F4805F0CD1636D43F00103636507E0636D43F010036365A36D43F00103D5
S32508004F60A3652046FEF7E8FE23680C221A6016F0200F02D015F0200F05D116F0400F4CD025
S32508004F8015F0400F49D0636D13F0100F03D1636D43F4005363652368DA6C12F0C00F2AD111
S32508004FA00121DA6812F4406F27D10120DA6871B312F0007F03D050B312F4005F27D1196816
S32508004FC011F0400F23D012F4001F20D19A6812F0080F14D15A6822F060025A60636D23F493
S32508004FE080536365636D13F4807F10D1636D43F0010363650BE00021D3E70020D6E7636D0F
S3250800500043F010036365A36D43F00103A365204600F072FC236860221A6016F0800F02D073
S3250800502015F0800F2DD116F4807F02D015F4807F32D116F4007F02D015F4007F38D116F0F8
S32508005040100F17D015F0100F14D0636B23B12368DB6813F0010F0AD0636D43F48063636525
S32508005060A36D43F00203A3652046FEF779FE236810221A6016F4806F02D015F4806F23D112
S3250800508070BD636D43F4803363652046FFF711FF236880221A60C6E7636D43F40033636591
S325080050A0204600F02BFC23684FF480721A60C0E7636D43F480236365204600F020FC236815
S325080050C04FF400721A60BAE7636D43F480436365A36D43F00803A36523684FF480621A60E0
S325080050E0204600F00AFCCBE708B50346806A426D12F0500F30D1436D43F400734365036826
S325080051001A6812F0080F14D0DA6812F4406F20D1DB6813F4005F1CD1436D23F48073436522
S32508005120436D13F4805F14D1436D43F0010343650FE0DB6813F0020F0BD1436D23F480737B
S325080051404365436D13F4805F03D1436D43F001034365FEF7F1FD08BD426D12F0100F04D153
S32508005160C26C526B18469047F5E7FEF7F9FDF2E708B5806A436D43F040034365836D43F0C9
S3250800518004038365FEF7ECFD08BD0000F0B583B00022019290F85020012A00F03F820346C5
S325080051A0012280F850200268926812F0040F09D0426D42F0200242650120002283F85020AC
S325080051C003B0F0BD4A68052A08D8023A032A68D8DFE802F0025D60630C224A601D684C680B
S325080051E03035220A920002F00C02A85804F01F0E1F2404FA0EF420EA04000C68C4F3846CF1
S325080052000CFA0EFC40EA0C00A8501C68A26812F0040200D00122A06810F0080000D00120B8
S325080052200AB9002840D01868826812F0010F17D10A68CD68D0F8B040C2F3120C24EA0C04B1
S3250800524005F0180CAE4D25FA0CF52A40C2F312022243C0F8B020C868AA4A904200F0B880CE
S325080052600A68A9490A4200F0D581A849896801F0E074A748824200F07F81A648824200F0BE
S32508005280A281A548824200F0B281002095E712224A60A3E718224A60A0E74FF480724A60BB
S325080052A09CE706224A6099E70E688D681434720E920002F00402A058C6F3045C072606FA10
S325080052C00CF620EA060005FA0CF52843A0504C691868C268C2F3C102520094400D69042DAF
S325080052E00ED00E68603050F825708C4A3A4006F0F8463443224342F0004240F8252092E715
S32508005300026E046EC4F384640A68C2F3120585BBC2F38462944234D01C68626E606EC0F336
S3250800532084600A68C2F3120585BBC2F38462904234D01C68A26EA06EC0F384600A68C2F32C
S32508005340120585BBC2F38462904234D01C68E26EE06EC0F384600A68C2F3120585BBC2F38B
S32508005360846290427FF45FAFE26E22F00042E26659E792FAA2F212B1B2FA82F2CAE72022C4
S32508005380C8E7026E22F000420266C5E792FAA2F212B1B2FA82F2CAE72022C8E7626E22F0F1
S325080053A000426266C5E792FAA2F212B1B2FA82F2CAE72022C8E7A26E22F00042A266C5E76C
S325080053C092FAA2F212B1B2FA82F2CAE72022C8E71C680A68C2F31205002D3BD1900E013050
S325080053E000F01F0009288CBF00200120002869D0002D3ED1900E0130800600F0F840002D8C
S3250800540043D14FEA926C0CF1010C0CF01F0C012606FA0CF63043002D46D1920E013202F05D
S325080054201F0202EB4202120510438D6804F1140E420E920002F004025EF80240C0F304501D
S325080054400726864024EA060C85404CEA05054EF8025005E792FAA2F048B1B0FA80F0013040
S3250800546000F01F0009288CBF00200120BEE72020F5E792FAA2F030B1B0FA80F001308006C1
S3250800548000F0F840BBE72020F8E792FAA2F64EB1B6FA86F6013606F01F064FF0010C0CFA22
S325080054A006F6B7E72026F5E792FAA2F242B1B2FA82F2013202F01F0202EB42021205B3E7C7
S325080054C02022F6E765BB900E0130800600F0F84095BB4FEA926C0CF1010C0CF01F0C012623
S325080054E006FA0CF63043B5BB920E013202F01F0202EB42021E3A120542F00072104394E7C1
S32508005500FFFF070000007F400000088000030450000052C7000084CB0100008000F0FF03FF
S3250800552092FAA2F030B1B0FA80F00130800600F0F840CDE72020F8E792FAA2F64EB1B6FABF
S3250800554086F6013606F01F064FF0010C0CFA06F6C8E72026F5E792FAA2F25AB1B2FA82F205
S32508005560013202F01F0202EB42021E3A120542F00072C3E72022F3E711F4000F7FF47DAE1B
S325080055801968274A914201D0002016E644F400022448816821F0E0710A438260224A126845
S325080055A092092249A1FB02129209013202EB42029200019202E0019A013A0192019A002AF3
S325080055C0F9D10020F9E511F0807F7FF45AAE1968134A914201D00020EFE544F08072114885
S325080055E0816821F0E0710A4382600020E5E511F4800F11D119680A4A914201D00020DCE569
S3250800560044F480020748816821F0E0710A4382600020D2E50020D0E50020CEE50220CFE5A4
S3250800562000000450000304509C000020632D3E0530B583B00023019303689A6812F0010FD4
S3250800564058D1044699682D4A114219D19A6822F0004222F03F0242F001029A60284B9B68C6
S3250800566013F4000F1CD0274B1B689B09264AA2FB03239B09013303EB43039B0001930CE027
S32508005680436D43F010034365836D43F001038365012030E0019B013B0193019B002BF9D121
S325080056A0FFF7FAFA054623681A6812F0010F1FD19A6812F0010F07D19A6822F0004222F044
S325080056C03F0242F001029A60FFF7E6FA431B022BE9D923681B6813F0010FE4D1636D43F050
S325080056E010036365A36D43F00103A365012002E0002000E0002003B030BD00BF3F00008031
S32508005700000304509C000020632D3E0570B504460068806810F0040F4ED10E46154694F869
S325080057205030012B4AD0012384F850302046FFF77FFF00283CD1636D23F4706323F0010395
S3250800574043F480736365636D13F4805F2DD0A36D23F00603A365E36C194ADA62E36C194AC2
S325080057601A63E36C184A5A6323681C221A60002384F850302268536843F010035360226806
S32508005780D36843F00103D36021682B4632464031E06C00F007FF2268936823F0004323F043
S325080057A03F0343F00403936007E00023A365D2E7002384F8503000E0022070BD0220FCE74E
S325080057C0E9500008A94E00087151000838B504460268936813F0020300D00123916811F01F
S325080057E0010F39D0002B39D1936803F00D03012B09D0636D43F010036365A36D43F0010325
S32508005800A365012029E0936823F0004323F03F0343F002039360236803221A60FFF73CFA21
S32508005820054623689B6813F0010F13D0FFF734FA401B0228F5D923689B6813F0010FF0D0B3
S32508005840636D43F010036365A36D43F00103A365012002E0002000E0002038BD0020FCE7F2
S3250800586030B583B00023019390F85030012B41D004460D46012380F85030FFF7A7FF80BB76
S32508005880636D23F4885323F0020343F0020363652268936823F0404323F03F0305F08045F6
S325080058A02B4343F00043936023689B68002B06DB636D23F0030343F00103636515E0019BF0
S325080058C001330193019BB3F5912FEDD3636D23F0120343F010036365002384F850300120E8
S325080058E006E0636D43F010036365002384F8503003B030BD0220FBE7704770477047704737
S325080059007047002800F0A18038B5044690F82030D3B12268136843F001031360FFF7BCF99C
S32508005920054623685A6812F0010F10D1FFF7B4F9401B0A28F5D9636A43F4003363620523AC
S3250800594084F82030012038BDFEF7A4FFE1E71A6822F002021A60FFF79FF9054623685A68BF
S3250800596012F0020F0DD0FFF797F9401B0A28F5D9636A43F400336362052384F82030012037
S32508005980E1E7227E012A3DD01A6822F080021A60637E012B3BD02268136823F040031360E3
S325080059A0A37E012B39D02268136823F020031360E37E012B37D02268136843F01003136083
S325080059C0237F012B35D02268136823F008031360637F012B33D02268136823F004031360AD
S325080059E0A368E268134322691343626913436268013A21681343CB6100206062012384F85A
S32508005A002030A0E71A6842F080021A60C0E72268136843F040031360C2E72268136843F07B
S32508005A2020031360C4E72268136823F010031360C6E72268136843F008031360C8E72268DD
S32508005A40136843F004031360CAE701207047026890F82030013BDBB2012B05D9436A43F48E
S32508005A60802343620120704730B4D2F8003243F00103C2F800324B6903F01F03012000FA11
S32508005A8003F3D2F81C026FEA030C20EA0300C2F81C02C869B0B9D2F80C020CEA0000C2F8AB
S32508005AA00C028C884869CD6844EA0544483042F830400C8848698D6844EA0544483002EB21
S32508005AC0C0004460C86901281BD0886980BBD2F804020CEA0000C2F80402086970BBD2F8F7
S32508005AE014020CEA0000C2F81402096A01292BD0D2F8003223F00103C2F80032002030BC19
S32508005B007047D2F80C021843C2F80C028C8848690D6844EA0544483042F830408C8948692C
S32508005B208D6844EA0544483002EBC0004460CCE7D2F804021843C2F80402CEE7D2F81402EF
S32508005B401843C2F81402D0E7D2F81C120B43C2F81C32CDE770B5044690F82050EDB2012D1F
S32508005B6006D0436A43F4002343620125284670BD022380F820300268136823F00103136078
S32508005B80FFF78AF8064623685B6813F0010F0CD0FFF782F8831B0A2BF5D9636A43F40033AE
S32508005BA06362052384F82030E0E700256562DDE730B590F820C00468A4680CF1FF3C5FFA51
S32508005BC08CFCBCF1010F62D814F0E05F59D0C4F3016C012404FA0CF41C608B68002B3DD1DD
S32508005BE00D68CB68046843EA45550CF118031B01E55003680C690CF1180E03EB0E135C6085
S32508005C000B7D012B35D0D17993791B0443EA0163517943EA012314790168234301EB0C1137
S32508005C20C1F88C31D17893781B0443EA0163517843EA0123117802680B4302EB0C12C2F8BC
S32508005C40883102680CF1180C4FEA0C1C52F80C3043F0010342F80C3000201DE04C6843EA60
S32508005C60C403CC6823430CF11804240105682B51BFE7036803EB0E13596841F480715960CE
S32508005C80C1E7436A43F400134362012004E0436A43F480234362012030BD90F820C00CF10E
S32508005CA0FF3C5FFA8CFCBCF1010F00F2958030B451B90468E46814F0030F10D1436A43F475
S32508005CC000134362012077E00468246914F0030F05D1436A43F40013436201206CE001F1A6
S32508005CE01B04240105682C5904F004049460002C64D101F11B04240105682C59640D146002
S32508005D00046801F11B0C4FEA0C1C54F80C4004F00204D46004686444646804F00F0414616D
S32508005D20046864446468C4F307249461046864446468240C5461026802EB0112D2F8B821CC
S32508005D401A70026802EB0112D2F8B821C2F307225A70026802EB0112D2F8B821C2F30742EB
S32508005D609A70026802EB0112D2F8B821120EDA70026802EB0112D2F8BC211A71026802EBA1
S32508005D800112D2F8BC21C2F307225A71026802EB0112D2F8BC21C2F307429A71026802EB21
S32508005DA00112D2F8BC21120EDA7179B90268D36843F02003D360002030BC704701F11B047C
S32508005DC0240105682C59E408546099E70268136943F020031361EEE7436A43F480234362CD
S32508005DE00120704790F82030013BDBB2012B05D9436A43F4802343620120704702685369E8
S32508005E000B43536100207047704770477047704770477047704770477047704770472DE9A8
S32508005E20F84F054603685C69D3F804809F68D3F80CB0D3F810A0D3F8189014F001063BD0B1
S32508005E4017F0010616D001229A6017F0020F08D117F0040F0CD117F0080606D04FF4805637
S32508005E6008E0FFF7D1FF002604E0FFF7D0FF01E04FF4006617F4807F0DD02B684FF480725E
S32508005E809A6017F4007F40F0868017F4806F00F0868046F4005617F4803F0DD02B684FF43D
S32508005EA080329A6017F4003F40F0838017F4802F00F0838046F4004614F0080F07D01BF081
S32508005EC0100F04D046F400762B681022DA6014F0040F02D01BF0080F79D114F0020F04D0D4
S32508005EE02B68DB6813F0030F78D114F0400F07D01AF0100F04D046F480662B6810221A61D9
S32508005F0014F0200F02D01AF0080F6BD114F0100F04D02B681B6913F0030F6AD114F4003F6C
S32508005F2002D018F0100F68D114F4803F02D018F0080F69D114F4004F7AD018F0040F74D02F
S32508005F4014F4807F04D019F0010F01D046F0010614F4007F04D019F0020F01D046F00206AD
S32508005F6014F4806F04D019F0040F01D046F0040614F4006F59D019F0700956D0B9F1400FDA
S32508005F8065D058D8B9F1200F5ED0B9F1300F42D146F0200644E02846FFF737FF7BE717F404
S32508005FA0006F02D046F4804675E72846FFF730FF71E72846FFF72AFF7EE717F4002F02D04D
S32508005FC046F4803678E72846FFF723FF74E72B680822DA602846FFF71DFF7EE72846FDF745
S32508005FE069FF82E72B6808221A612846FFF714FF8CE72846FFF70FFF90E72B6810225A6038
S325080060002846FFF70AFF8FE72B6808225A602846FFF704FF8EE7B9F1100F01D146F008065D
S325080060202A68936923F0700393612B6804225A609EB9BDE8F88FB9F1500F0BD0B9F1600F57
S32508006040EED146F48076EBE746F01006E8E746F04006E5E746F08006E2E76B6A33436B6271
S325080060602846FDF749FFE4E7074AD36823F4E0631B041B0C000200F4E060034343F0BF63A0
S3250800608043F40033D360704700ED00E000B5194BDB68C3F30223C3F1070CBCF1040F28BF2C
S325080060A04FF0040C03F1040EBEF1060F18D9033B4FF0FF3E0EFA0CFC21EA0C0199400EFA05
S325080060C003FE22EA0E020A4300280BDB1201D2B200F1604000F5614080F800235DF804FB8D
S325080060E00023E5E700F00F001201D2B2024B1A54F4E700BF00ED00E014ED00E0002807DB00
S3250800610000F01F02400901239340024A42F82030704700BF00E100E0BFF34F8F0549CA6803
S3250800612002F4E062044B1343CB60BFF34F8F00BFFDE700BF00ED00E00400FA050138B0F1AD
S32508006140807F0BD24FF0E0235861054AF02182F823100020986107221A6170470120704701
S3250800616000ED00E070B110B50446037933B102232371002020610123237110BD4371FEF72C
S32508006180DDFBF4E7012070474279012A2CD010B4034601224271022018711C68206801F0F9
S325080061A0100C02FA0CF20243226089B919680A6802F03C02042A06D001221A7100205871F4
S325080061C05DF8044B70474A6842F001024A60F3E719680A6802F47012B2F5802FECD14A68BB
S325080061E042F002024A60E7E70220704710B483B0002401940068019051B901990A44083235
S325080062000192019A1360002003B05DF8044B704701990A4414320192F3E7F8B54379012B71
S3250800622000F0948004460D46164601234371022303710B68042B32D02B69012B79D02068AD
S32508006240C16B06F010020723934021EA03012B68AE683343EE68334393400B43C363206836
S3250800626003684FF48041914023EA010303602068016840F6FC73934021EA03016B6893403E
S325080062800B43036020680368C02101FA02F223EA020303600123237100206071F8BDFEF7B4
S325080062A0FBFC07467EB123685B6B002B3ADAFEF7F3FCC01B0128F6D9236943F008032361C8
S325080062C003202071EAE723685B6B13F4004F0BD0FEF7E2FCC01B0128F5D9236943F008033A
S325080062E0236103202071D9E70120FEF7DBFC2368AA691A642068836C06F0100240F2FF31AE
S32508006300914023EA0103E96991400B4383642068C36CFF21914023EA0103296A91400B43CA
S32508006320C36489E70120FEF7BDFC2368AA695A64E0E721688A6B06F010001F23834022EA31
S3250800634003026B69834013438B6378E70220A5E7002800F083802DE9F04F83B08946044686
S325080063600379DBB2022B7BD04379012B7AD0012141710068C56B02F010070723BB4005EAD3
S32508006380030B0568B94025EA010101602068C16B6FEA030A21EA0303C3632368019392B94E
S325080063A0019B08330193019B4FF400621A60226813684FF4804808FA07F843EA08031360ED
S325080063C00825102605E0019B14330193EBE72E446D089DB121688B6B1F22BA4023EA02031D
S325080063E006FA07F213438B630120FEF75BFC23685B6B38EA0303EAD1761BE9E721688B6BD1
S325080064001F22BA40D54323EA020306FA07F213438B630120FEF746FC23685A6B18EA020F11
S3250800642006D101369A6B154006FA07F73D439D632268136823EA08031360C9F8146001237F
S32508006440C9F810302268D36B0AEA030A4AEA0B03D3630020607103B0BDE8F08F012070474C
S325080064600120F8E70220F6E730B4446C04F01C0C012404FA0CF4056C6C60046863608368E5
S32508006480102B05D0036899600368DA6030BC704703689A600368D960F8E70000002873D0DF
S325080064A010B403460068394A90424AD8384A02443849A1FB0212120992005A64364A1A6480
S325080064C0022283F82520016821F4FF4121F070019A68DC6822431C6922435C6922439C69C6
S325080064E02243DC6922431C6A22430A4302609A68B2F5804F1BD0196C274A91422CD0264A4D
S32508006500D2F8A814586C00F01C0C0F2000FA0CF021EA0001C2F8A814D2F8A81458685C6C56
S3250800652004F01C0C00FA0CF00143C2F8A8140020D863012283F8252083F824005DF8044B00
S325080065407047164A02441349A1FB0212120992005A64134A1A64B3E7D2F8A810586C00F0AE
S325080065601C0C0F2000FA0CF021EA0001C2F8A810D2F8A81058685C6C04F01C0C00FA0CF026
S325080065800143C2F8A810D2E70120704707040240F8FFFDBFCDCCCCCC00000240F8FBFDBF84
S325080065A00004024038B5044690F82400012832D0012084F8240094F82500C0B2012804D098
S325080065C0002384F82430022038BD022084F825000020E0632568286820F001002860204661
S325080065E0FFF742FF236B5BB12268136843F00E0313602268136843F0010313600020E3E767
S325080066002268136823F0040313602268136843F00A031360EDE70220D6E708B590F82530D5
S32508006620DBB2022B03D00423C363012008BD0268136823F00E0313600268136823F0010314
S325080066401360436C03F01C03016C012202FA03F34B6080F82520002380F82430836B13B16D
S3250800666098470020E2E70020E0E738B5036C196804682568436C03F01C0304229A400A427A
S3250800668015D015F0040F12D0236813F0200F03D1236823F004032360436C03F01C02016C27
S325080066A0042393404B60036B03B1984738BD02229A400A421CD015F0020F19D0236813F06E
S325080066C0200F06D1236823F00A032360012380F82530436C03F01C02016C022393404B60B7
S325080066E0002380F82430C36A002BDFD09847DDE7082202FA03F30B42D8D015F0080FD5D021
S32508006700236823F00E032360436C03F01C03016C012202FA03F34B60C26380F82520002346
S3250800672080F82430436B002BC0D09847BEE70000F0B583B0002362E085685E000324B440EF
S3250800674025EA0405CC68B4402C438460456825EA0C054C68C4F300149C402C4344605FE01E
S32508006760DD08083550F8254003F0070C4FEA8C0C4FF00F0E0EFA0CFE24EA0E0E0C6904FA5A
S325080067800CF444EA0E0440F8254060E0022400E0002404FA0EF42C430CF1020C4C4D45F854
S325080067A02C404C4CA568D44325EA02064F6817F4801F01D042EA0506464DAE60ED6804EA3F
S325080067C005064F6817F4001F01D042EA0506414DEE606D6804EA05064F6817F4003F01D03B
S325080067E042EA05063B4D6E602D682C404E6816F4803F01D042EA0504364A146001330A68DE
S3250800680032FA03F462D04FF0010C0CFA03FC1CEA0202F3D04C6804F00304013C012C8BD97A
S325080068204C6804F00304032C0CD0C4685D004FF0030C0CFA05FC24EA0C0C8C68AC4044EA7E
S325080068400C04C4604C6804F00304022C88D004684FEA430E4FF0030C0CFA0EFC24EA0C0C47
S325080068604C6804F0030404FA0EF444EA0C0404604C6814F4403FC1D0174C256E45F00105BC
S325080068802566246E04F001040194019C4FEA930C0CF102050E4C54F8255003F0030E4FEA6E
S325080068A08E0E0F2404FA0EF425EA0405B0F1904F3FF46EAF094CA04206D004F58064A04247
S325080068C03FF464AF072464E7012462E703B0F0BD00000140000401400010024000040048FC
S325080068E00369194201D001207047002070470AB18161704781627047436901EA030221EAAE
S32508006900030141EA024181617047002859D010B5044690F84130002B43D0242384F8413093
S325080069202268136823F0010313606368226823F0706313612268936823F400439360E368EE
S32508006940012B33D0A368226843F404439360E368022B31D02268536843F0007343F4004316
S3250800696053602268D36823F40043D360236962691343A169226843EA0123D360E369216A68
S3250800698022680B4313602268136843F00103136000206064202384F84130206384F842009A
S325080069A010BD80F84030FDF7F9FFB6E7A368226843F400439360CAE723684FF400625A60EE
S325080069C0C8E701207047034690F84120D2B2202A23D190F84020012A21D0012280F840202F
S325080069E0242280F841200068026822F0010202601868026822F480520260186802681143AF
S32508006A00016019680A6842F001020A60202283F84120002083F840007047022070470220CA
S32508006A207047034690F84120D2B2202A21D190F84020012A1FD0012280F84020242280F8E4
S32508006A4041200068026822F0010202601868026822F4706242EA0122026019680A6842F0D6
S32508006A6001020A60202283F84120002083F840007047022070470220704700282FD038B525
S32508006A80044603684CF6CC421A60036845F255521A60036842685A60036882689A60FEF793
S32508006AA0FBF805462368DA6812F0070F0BD0FEF7F3F8401B3128F5D92368DB6813F0070F81
S32508006AC0F0D0032005E01969E268914202D01A61002038BD4AF6AA221A600020F9E7012038
S32508006AE0704703684AF6AA221A60002070470000024B186800F4C060704700BF0070004002
S32508006B00B0F5007F0FD01F4B1B6803F4C063B3F5806F34D01B4A136823F4C06343F480638E
S32508006B20136000207047174B1B6803F4C063B3F5007F20D0134A136823F4C06343F400732B
S32508006B401360114B1B68322202FB03F30F4AA2FB03239B0C013300E0013B0A4A526912F466
S32508006B60806F01D0002BF7D1064B5B6913F4806F03D10020704700207047032070470020CD
S32508006B80704700BF007000409C00002083DE1B4330B583B00446204B9B6D13F0805F0BD0B4
S32508006BA0FFF7A6FFB0F5007F17D0802C1FD82DD0702C2DD000211BE0174DAB6D43F080534A
S32508006BC0AB65AB6D03F080530193019BFFF790FFAB6D23F08053AB65E4E7802C03D9A02CD7
S32508006BE003D9022104E0002102E0012100E003210A4A136823F007030B431360136803F060
S32508006C0007038B4206D1002003B030BD0221EFE70121EDE70120F7E7001002400020024056
S32508006C20284A9368D26802F0030213F00C030AD00C2B06D0042B1FD0082B20D00020024606
S32508006C4010E0012AF6D11F4A126812F0080F0CD11C4AD2F89420C2F303221B4951F82220BE
S32508006C6043B100200C2B0DD07047164A1268C2F30312F2E71046F5E714480022F2E71448C5
S32508006C800022EFE70F4BDB6803F00303022B16D0032B00D10E4A0B49CB68C3F30213013368
S32508006CA0C868C0F3062002FB00F0B0FBF3F0CB68C3F3416301335B00B0FBF3F0D4E7034A90
S32508006CC0E9E700BF0010024068B500080024F400005A6202002800F01C83F0B583B00446F1
S32508006CE0964B9D6805F00C05DE6806F00306036813F0100F5AD0E5B10C2D18D0A369002BB0
S32508006D0000F0BB808D4A136843F001031360FDF7C3FF0746894B1B6813F0020F40F09A8086
S32508006D20FDF7BAFFC01B0228F4D90320FCE2012EE4D1824B1B6813F0020F03D0A369002B73
S32508006D4000F0E982206A7D4B1B6813F0080F5BD07A4B1B6803F0F00398425CD8774B1A6830
S32508006D6042F008021A601A6822F0F002216A0A431A605A6822F47F42E16942EA01225A608B
S32508006D80002D60D0FFF74CFF6C4B9B68C3F303136B4AD35C03F01F03D8406A4B18606A4BCE
S32508006DA01868FDF735FF002840F0BE82236813F0010F00F08180082D75D00C2D71D0636837
S32508006DC0B3F5803F00F09780B3F5A02F00F099805A4B1A6822F480321A601A6822F4802214
S32508006DE01A606368002B00F09980FDF755FF0746524B1B6813F4003F5ED1FDF74DFFC01BC7
S32508006E006428F5D903208FE24C4BD3F894301B0903F0F003A0E7FFF7BBFE002840F07D82B9
S32508006E20464B1A6842F008021A601A6822F0F002216A0A431A605A6822F47F42E16942EA94
S32508006E4001225A609EE7206AFFF7A2FE002899D0012069E2394B1A6842F008021A601A6867
S32508006E6022F0F002216A0A431A605A6822F47F42E16942EA01225A6098E7304A136823F03B
S32508006E8001031360FDF708FF07462C4B1B6813F0020F8BD0FDF700FFC01B0228F5D90320D3
S32508006EA042E2032E8BD1254B1B6813F4003F03D06368002B00F03382236813F0020F58D0A5
S32508006EC0042D45D00C2D41D0E368002B77D01B4A136843F480731360FDF7DEFE0646174B5C
S32508006EE01B6813F4806F61D1FDF7D6FE801B0228F5D9032018E2114A136843F4803313602E
S32508006F006FE703F18043A3F53C331A6842F480221A601A6842F480321A6062E7FDF7BCFEA0
S32508006F200746064B1B6813F4003FC5D0FDF7B4FEC01B6428F5D90320F6E100BF0010024061
S32508006F4058B500089C000020A4000020022EBBD1A44B1B6813F4806F03D0E368002B00F031
S32508006F60E081A04A536823F0F853216943EA01635360236813F0080F4CD063699BB3994A13
S32508006F80D2F8943043F00103C2F89430FDF784FE0646944BD3F8943013F0020F3AD1FDF75D
S32508006FA07BFE801B0228F4D90320BDE18D4A536823F0F853216943EA01635360D9E7894AA6
S32508006FC0136823F480731360FDF766FE0646854B1B6813F4806FCCD0FDF75EFE801B02280D
S32508006FE0F5D90320A0E17F4AD2F8943023F00103C2F89430FDF750FE06467A4BD3F8943043
S3250800700013F0020F06D0FDF747FE801B0228F4D9032089E1236813F0040F7AD0714B9B6D71
S3250800702013F0805F36D16F4B9A6D42F080529A659B6D03F080530193019B01266A4B1B6838
S3250800704013F4807F28D0A368012B39D0052B3FD0644BD3F8902022F00102C3F89020D3F830
S32508007060902022F00402C3F89020A368002B3DD0FDF712FE07465B4BD3F8903013F0020FF6
S3250800708046D1FDF709FEC01B41F288339842F2D9032049E10026D1E7534A136843F48073F5
S325080070A01360FDF7F9FD07464F4B1B6813F4807FC9D1FDF7F1FDC01B0228F5D9032033E16F
S325080070C0484AD2F8903043F00103C2F89030CCE7444BD3F8902042F00402C3F89020D3F8AA
S325080070E0902042F00102C3F89020BEE7FDF7D4FD07463C4BD3F8903013F0020F08D0FDF789
S32508007100CBFDC01B41F288339842F2D903200BE1E6B9236813F0200F35D0636AE3B1314ADF
S32508007120D2F8983043F00103C2F89830FDF7B4FD06462C4BD3F8983013F0020F23D1FDF7FF
S32508007140ABFD801B0228F4D90320EDE0254A936D23F080539365DCE7224AD2F8983023F0D6
S325080071600103C2F89830FDF797FD06461D4BD3F8983013F0020F06D0FDF78EFD801B02287E
S32508007180F4D90320D0E0A36A002B00F0CC80022B17D00C2D00F0CC80124A136823F0807367
S325080071A01360FDF779FD04460E4B1B6813F0007F00F0A880FDF770FD001B0228F4D903208E
S325080071C0B2E0084BDB6803F00301E26A91420DD00C2D00F0AB80034B1B6813F0806F2FD070
S325080071E00120A1E0001002400070004003F07002216B0139B2EB011FEAD103F4FE42616B37
S32508007200B2EB012FE4D103F07842A16BB2EBC16FDED103F4C001E26B5208013AB1EB425FD2
S32508007220D6D103F0C063226C5208013AB3EB426FCED1404B1B6813F0007F49D0002073E056
S325080072403C4A136823F080731360FDF725FD0546384B1B6813F0007F06D0FDF71DFD401B7E
S325080072600228F5D903205FE0324AD36832491940E36A206B013843EA0013606B43EA0023AF
S32508007280E06B4008013843EA4053206C4008013843EA4063A06B43EAC0631943D160136814
S325080072A043F080731360D36843F08073D360FDF7F3FC04461F4B1B6813F0007F06D1FDF72C
S325080072C0EBFC001B0228F5D903202DE000202BE0184B1A6842F080721A60DA6842F0807262
S325080072E0DA60FDF7D9FC0446124B1B6813F0007F06D1FDF7D1FC031B022BF5D9032013E00A
S32508007300002011E00B4AD1680C4B0B40D36000200AE001207047012006E0012004E00120DC
S3250800732002E0012000E0002003B0F0BD0120FBE70120F9E7001002408C809D01FCFFEEFEF5
S32508007340002800F0AF8070B50D460446594B1B6803F007038B420BD2564A136823F0070310
S325080073600B431360136803F007038B4240F09C80236813F0020F0CD0A2684F4B9B6803F098
S32508007380F0039A4205D94C498B6823F0F0031A438A60236813F0010F39D06368032B09D0E4
S325080073A0022B26D063BB444A126812F0020F06D1012076E0404A126812F0007F76D03E49C3
S325080073C08A6822F0030213438B60FDF765FC0646394B9B6803F00C036268B3EB820F16D04C
S325080073E0FDF75AFC801B41F288339842F0D9032057E0314A126812F4003FE0D1012050E073
S325080074002D4A126812F4806FD9D1012049E0236813F0020F0CD0A268274B9B6803F0F003A4
S325080074209A4205D224498B6823F0F0031A438A60204B1B6803F00703AB420AD91D4A136841
S3250800744023F007032B431360136803F00703AB422ED1236813F0040F06D0174A936823F4D2
S32508007460E063E1680B439360236813F0080F07D0114A936823F46053216943EAC103936027
S32508007480FFF7CEFB0C4B9B68C3F303130B4AD35C03F01F03D8400A4B18600A4B1868FDF7B2
S325080074A0B7FB70BD012070470120FAE70120F8E70120F6E7002002400010024058B500083E
S325080074C09C000020A4000020F8B504460F46584BDB6813F0030F18D0554BDB6803F0030313
S325080074E00268934202D001252846F8BD002A00F09D804F4BDB68C3F3021301334268934292
S3250800750001D00125F0E7002509E00368022B56D0032B5BD0012B41D00125002DE4D1444A97
S32508007520136823F080631360FDF7B6FB0646404B1B6813F0006F05D0FDF7AEFB831B022BAB
S32508007540F5D90325002DCFD1002F4DD138490B6923F0784323F4FE43A068E268D20642EA9C
S32508007560002213430B61324A136843F080631360FDF792FB06462E4B1B6813F0006F05D188
S32508007580FDF78AFB831B022BF5D90325002DABD1274A1369A1690B431361A5E7244A1268CD
S325080075A012F0020F1ED02248C26822F073026168013943EA01131343C3600025ADE71C4AC5
S325080075C0126812F4806FEED10125A6E7184A126812F4003FE7D1164A126812F4802FE2D1A1
S325080075E001259AE7012598E7012F0FD01048026922F0C06222F4FE42A16863695B08013B61
S325080076005B0643EA01231A430261ACE70848026922F4C00222F4FE42A16823695B08013B3A
S325080076205B0543EA01231A4302619CE701255BE7001002402DE9F04182B00446036813F459
S32508007640006F25D0C36BB3F5000F06D0B3F5400F12D04BB1012637461CE0AE4AD36843F41E
S325080076608033D360002708E000210430FFF72CFF074610B106460DE00027A64AD2F88830B1
S3250800768023F44003E16B0B43C2F88830002601E000263746236813F4003F6BD09D4B9B6DD0
S325080076A013F0805F4CD19B4B9A6D42F080529A659B6D03F080530193019B4FF00108964AA7
S325080076C0136843F480731360FDF7E6FA0546924B1B6813F4807F05D1FDF7DEFA401B0228D8
S325080076E0F5D90327002F40D18A4BD3F8903013F4407315D0226D9A4212D0864AD2F890309E
S3250800770023F44073D2F8901041F48031C2F89010D2F8901021F48031C2F89010C2F89030E3
S3250800772013F0010F0FD1002F40F0C980794AD2F8903023F44073216D0B43C2F8903015E03E
S325080077404FF00008BBE7FDF7A7FA0546714BD3F8903013F0020FE6D1FDF79EFA401B41F226
S3250800776088339842F2D90327DDE73E46B8F1000F40F0A780236813F0010F08D0654AD2F82B
S32508007780883023F00303216A0B43C2F88830236813F0020F08D05F4AD2F8883023F00C03FB
S325080077A0616A0B43C2F88830236813F0200F08D0584AD2F8883023F44063A16A0B43C2F8AA
S325080077C08830236813F4007F08D0524AD2F8883023F44023616B0B43C2F88830236813F444
S325080077E0806F08D04B4AD2F8883023F44013A16B0B43C2F88830236813F0400F08D0454A23
S32508007800D2F8883023F44053E16A0B43C2F88830236813F4807F08D03E4AD2F8883023F499
S325080078204033216B0B43C2F88830236813F4005F0FD0384AD2F8883023F04063216C0B4316
S32508007840C2F88830236CB3F1006F40D0B3F1806F42D0236813F4802F0FD02E4AD2F8883037
S3250800786023F04063616C0B43C2F88830636CB3F1006F39D0B3F1806F3BD0236813F4804FCD
S325080078800CD0244AD2F8883023F04053A16C0B43C2F88830A36CB3F1805F32D0236813F475
S325080078A0004F08D01B4AD2F8883023F08043E16C0B43C2F88830304602B0BDE8F0813E4607
S325080078C054E7144A936D23F08053936552E7D36843F48013D360BCE70121201DFFF7F4FDC9
S325080078E00028B6D00646B4E7D36843F48013D360C3E70121201DFFF7E7FD0028BDD00646C9
S32508007900BBE70221201DFFF7DFFD0028C6D00646C4E700BF00100240007000402DE9F047C2
S3250800792082B00546884617461E46FDF7B5F90A9B1B1A03EB0609FDF7AFF982462A4B1B6858
S32508007940C3F3CB3309FB03F301932B689C6838EA04040CBF01230023BB4240D0B6F1FF3F12
S32508007960F3D0FDF799F9A0EB0A0048450AD2B9F1000F07D0019A02B14A46019B013B0193D8
S325080079809146E2E72A68536823F0E00353606B68B3F5827F0BD0AB6AB3F5005F14D00123C8
S325080079A085F85D30002385F85C30032018E0AB68B3F5004F02D0B3F5806FECD12A6813682B
S325080079C023F040031360E6E72A68136823F4005313602A68136843F400531360DFE7002029
S325080079E002B0BDE8F08700BF9C0000202DE9F04782B006460C4615461F4600238DF8033078
S32508007A00FDF74AF90A9B1B1A03EB0708FDF744F98146D6F800A0314B1B6803EB8303C3EBC3
S32508007A20C3031B0D08FB03F3019302E0B7F1FF3F12D133689B6803EA040CAC454AD0B4F5C3
S32508007A40C06FF3D1002DF1D19AF80C30DBB28DF803309DF80330E9E7FDF71EF9A0EB0900EC
S32508007A6040450AD2B8F1000F07D0019A02B14246019B013B01939046DBE73268536823F0C6
S32508007A80E00353607368B3F5827F0BD0B36AB3F5005F14D0012386F85D30002386F85C307F
S32508007AA0032018E0B368B3F5004F02D0B3F5806FECD13268136823F040031360E6E7326820
S32508007AC0136823F4005313603268136843F400531360DFE7002002B0BDE8F0879C000020BE
S32508007AE070B582B004460D46164600920B4600224FF4C051FFF77AFFB0B900962B460022CE
S32508007B0080212046FFF70AFFA8B900962B4600224FF4C0612046FFF769FF50B1236E43F0DA
S32508007B2020032366032004E0236E43F020032366032002B070BD236E43F02003236603207F
S32508007B40F7E770B582B004460D4616464368B3F5827F0DD000962B46002280212046FFF792
S32508007B60DDFE90B96368B3F5827F14D002B070BD8368B3F5004F02D0B3F5806FEAD122680C
S32508007B80136823F040031360E4E7236E43F0200323660320EAE7A368B3F5004F02D0B3F5E8
S32508007BA0806FE3D100962B4600224FF4C0612046FFF71CFF0028D9D0236E43F020032366CF
S32508007BC00320D3E700286AD010B50446436A33B94368B3F5827F05D00023C36102E000233B
S32508007BE0036143610023A36294F85D30002B4DD0022384F85D302268136823F040031360EA
S32508007C00E368B3F5E06F47D90022B3F5706F04D0B3F5E06F01D00023A362636803F48273D0
S32508007C20A16801F404410B43216901F002010B43616901F001010B43A16901F400710B4310
S32508007C40E16901F038010B43216A01F080010B43A16A01F4005120680B430360638B03F09E
S32508007C600403616A01F010010B43616B01F008010B43E16801F470610B4321681A434A60D3
S32508007C8000202066012384F85D3010BD84F85C302046FCF7C7FEABE74FF48052B5E70120AC
S32508007CA07047000038B5044690F85C00012800F0F780012084F85C0094F85D00C0B2656833
S32508007CC001280AD0B5F5827F40F0DB80A568002D40F0DC80042840F0DB80002900F0DA806D
S32508007CE0002A00F0D980002B00F0D88094F85D00C0B2042802D0052084F85D000020206693
S32508007D00A163A387E3872264A4F84430A4F84630E06420652268536823F4C0435360E368EF
S32508007D20B3F5E06F28D92268536823F48053536094F85D30DBB2042B69D0A36D594A1A631D
S32508007D40A36D594ADA62A36D584A5A63A36D00229A632168B4F846309BB2226C0C31A06DB8
S32508007D60FEF720FC002859D0236E43F010032366012084F85D0085E02268536843F4805385
S32508007D805360636D9B69B3F5806F1AD0A36D9B69B3F5806FCCD12268536823F480535360A3
S32508007DA0B4F8463013F0010F24D12268536823F400535360B4F84630C3F34E03A4F84630EE
S32508007DC0B6E7A38F13F0010F09D12268536823F480435360E38FC3F34E03E387D6E72268DD
S32508007DE0536843F480435360E38FC3F34E030133E387CBE72268536843F400535360B4F816
S32508007E004630C3F34E030133A4F8463090E7A36D274A1A63A36D274ADA6294E7226853689F
S32508007E2043F001035360626D00231363626DD362626D5363626D93632268E38F9BB20C320D
S32508007E40A16B606DFEF7AEFB98B923681A6812F0400F03D11A6842F040021A602268536865
S32508007E6043F0200353602268536843F00203536008E0236E43F010032366012084F85D0079
S32508007E8000E00220002384F85C3038BD0220F9E70220F7E70120F5E70120F3E70120F1E7BF
S32508007EA00220F2E7C77E0008637F0008D17E0008BB7E0008F37E0008704708B5806AFFF71D
S32508007EC0FBFF08BD704708B5806AFFF7FBFF08BD08B5806A0268536823F003035360036EB9
S32508007EE043F010030366012380F85D30FCF750F908BD38B50546846AFCF7CEFE2B681B68A0
S32508007F0013F0200F1FD1024621684B6823F020034B60A3681BB96368B3F5827F17D0216809
S32508007F204B6823F001034B6064212046FFF709FE08B1202323660023A4F84630012384F87C
S32508007F405D30236E4BB92046FCF710F938BD21684B6823F003034B60E6E72046FCF718F963
S32508007F60F4E738B50546846AFCF796FE2B681B6813F0200F1CD1024621684B6823F020037C
S32508007F804B6064212046FFF7ABFD18B1236E43F0200323662268536823F003035360002332
S32508007FA0E387A4F84630012384F85D30236E1BB92046FCF7C9F838BD2046FCF7E9F8FAE77B
S32508007FC010B584B0044602685168936803F04100012867D013F0020F02D011F0800F68D1EF
S32508007FE013F4B07F68D011F0200F65D013F0400F0FD094F85D00C0B203285FD0206E40F0FC
S325080080000400206600200090D068009090680090009813F0200F0CD0206E40F001002066DD
S325080080200020029090680290106820F040001060029A13F4807F09D0236E43F008032366EB
S325080080400023039323689B680393039B236E002B32D02268536823F0E0035360012384F84B
S325080080605D3011F0030F31D02268536823F003035360A36D4BB1174A9A63A06DFEF7CDFA0D
S3250800808018B1236E43F040032366636DA3B1114A9A63606DFEF7C1FA70B1236E43F0400358
S325080080A0236609E011F0400F94D0E36C2046984702E0236D2046984704B010BD0023019309
S325080080C0D368019393680193019BF5E72046FCF75FF8F1E7D980000808B5806A0023A0F871
S325080080E04630C387FCF754F808BD08B502F047FE10B102684068904708BD0000EFF30583E1
S325080081002BB9064B186828B901221A6070476FF0050070474FF0FF30704700BFF007002051
S32508008120EFF3058373B90A4B1B68012B0DD110B50024084BDC77064B02221A6001F0F4FE58
S32508008140204610BD6FF0050070474FF0FF307047F007002000ED00E008B5EFF3058343B997
S3250800816002F06AFA40B1022808D101F033FF002006E06FF0050003E0012001E04FF0FF30C7
S3250800818008BDF0B587B000240594EFF305847CBB70B32AB31568936903B918235C1E372C84
S325080081A04AD8546814F0010F48D1566976B14FEA960C946834B1D768B7F5C07F02D3176985
S325080081C007B1C6B92CB14FF0FF340EE04FF0800CEFE7D4688CB9146994B14FF0FF3404E0E3
S325080081E01546002418234FF0800C012C0AD0ACB1059807B0F0BD0124F7E74FF0FF34F4E737
S325080082000024F2E7146992680292019400930B466246294601F016FE0590E9E705AA01920C
S3250800822000930B461FFA8CF2294601F048FE0128DED000230593DBE70020DAE70020D8E7FB
S3250800824008B5EFF3058323B930B102F04FF8002008BD6FF00500FBE76FF00300F8E708B5CA
S32508008260EFF3058333B908B9002008BD01F0C8FF0020FAE76FF00500F7E700002DE9F043B0
S3250800828083B0EFF30587002F43D10646894615461C4600283FD0082000F04CFE804600288D
S325080082A03BD006604560B9F1000F00D0012704B32068A36813B1E2682B2A10D853B14FF011
S325080082C0FF33DBB10024404600F0B2FE204603B0BDE8F083E3687BB14FF0FF33F1E7019303
S325080082E00F4B009343463A46012102F093FB04460CE020460023E4E70023E2E7084B00937C
S3250800830043463A46012102F069FB0446002CDDD1D9E70024DAE70024D8E70446D6E700BF5C
S32508008320EB800008EFF305836BB90A4670B100B583B00093042102F097FB012809D1002076
S3250800834003B05DF804FB6FF0050070476FF0030070476FF00200F3E708B5EFF30583CBB9EE
S32508008360A0B1836813B1C2681F2A0BD82BB14FF0FF338BB900F04EFA08BDC36843B14FF0AD
S32508008380FF33F6E7184600F020FAF5E70023F0E70023EEE70020EFE70020EDE7F8B110B532
S325080083A082B00C4611F07F4F1CD1EFF305829AB10022019201AA00F049FBB8B1019BC3B1AE
S325080083C04FF0E0234FF08052C3F8042DBFF34F8FBFF36F8F204607E000F0EEFA04E06FF0A8
S325080083E0030070476FF0030002B010BD6FF00200FAE72046F8E770B5B0B10C46064611F028
S325080084007F4F14D1EFF3058353B100F0C7FA05462146304600F0B8FA58B96FF0020508E053
S3250800842000F08AFA054604E06FF0030501E06FF00305284670BD40B370B582B00C461D4642
S32508008440844611F07F4F23D1EFF3058323BB12F0010610D0012312F0020F0ED00022009584
S325080084602146604600F0E4F94EB1844312D0B5B16FF001000EE00023EDE70122EFE7044282
S3250800848008D17DB16FF0010004E06FF0030070476FF0030002B070BD6FF00500FAE76FF085
S325080084A00200F7E76FF00200F4E770B5EFF30583002B3FD1044600B1436813F0010600D048
S325080084C0012613F0080F38D14CB3A16811B1E3684F2B19D899B14FF0FF334BBB1EB304200E
S325080084E001F01DF805462DB104B124682146284601F0B0FAFDB1F6B145F001051BE0E368B8
S325080085007BB14FF0FF33E8E726B1042001F012F80546E8E7012001F00DF80546E3E7002382
S32508008520DBE70023D9E7012000F0F9FF0546DAE70025DFE70025284670BD0025FBE7EFF3DF
S325080085400582C2B910B503460C4620F0010003F0010398B13BB101F005FA012811D094B12F
S325080085606FF001000EE001F02AF901280ED07CB16FF0010006E06FF0050070476FF0030094
S3250800858000E0002010BD6FF00200FBE70020F9E76FF00200F6E7EFF30582B2B908B50346A5
S325080085A020F0010003F0010390B12BB100F0D1FF012810D1002008BD00231A46194600F007
S325080085C0DEFE01280AD10020F5E76FF0050070476FF00300EFE76FF00200ECE76FF00200C9
S325080085E0E9E770B582B0EFF30583002B3AD1144600283BD000293BD06AB393684BB1D26897
S325080086004F2A06D9226922B101FB00F56669AE421BD273B14FF0FF3363BB002200F08BFEAB
S32508008620054605B304B124682146284601F012FA19E0E3688BB9236913B14FF0FF33EBE7FB
S3250800864063696BB14FF0FF33E6E70025009500F028FE0546E5E70023DEE74FF0FF33DBE7E4
S325080086600023D9E70025284602B070BD0025FAE70025F8E70025F6E710B582B01C46EFF350
S325080086800583C3B118B329B33CBB0023019301AA00F07FFF012823D1019850B14FF0E02369
S325080086A04FF08052C3F8042DBFF34F8FBFF36F8F002002B010BDB0B1C1B10023224600F082
S325080086C05EFE012815D0B4B16FF00100F1E76FF00300EEE76FF00300EBE76FF00300E8E7E9
S325080086E06FF00200E5E76FF00300E2E76FF00300DFE70020DDE76FF00200DAE710B582B0EF
S325080087001C46EFF30583C3B110B321B334BB0023019301AA01F046F9012822D1019850B13D
S325080087204FF0E0234FF08052C3F8042DBFF34F8FBFF36F8F002002B010BDA8B1B9B12246E2
S3250800874000F08EFF012815D0B4B16FF00100F2E76FF00300EFE76FF00300ECE76FF0030013
S32508008760E9E76FF00200E6E76FF00300E3E76FF00300E0E70020DEE76FF00200DBE7000090
S32508008780034B0360034B0B6080231360704700BF700600206C040020034B0360034B0B6045
S325080087A04FF4807313607047F80B0020F40700201AB9084205D110467047814303D0002056
S325080087C07047012070470120704780B110B582B0044620230193019B202B11D04FF0500381
S325080087E083F31188BFF36F8FBFF34F8FFEE74FF0500383F31188BFF36F8FBFF34F8FFEE771
S32508008800002340F8043B00F02BF901232377204602B010BD38B5202000F08CFB044628B132
S32508008820002540F8045B00F01BF92577204638BD2DE9F84378B10C4616461D46074611F09A
S325080088407F4811D04FF0500383F31188BFF36F8FBFF34F8FFEE74FF0500383F31188BFF349
S325080088606F8FBFF34F8FFEE741B94FF0500383F31188BFF36F8FBFF34F8FFEE701F0DCFEEC
S3250800888050B9089B43B14FF0500383F31188BFF36F8FBFF34F8FFEE701F09CFBD7F800907D
S325080088A02A4621464846FFF783FFF0B116B129EA04033B6001F028FCB8F1000F12D048B900
S325080088C04FF0E0234FF08052C3F8042DBFF34F8FBFF36F8F01F0A4FF814610F0007F1AD047
S325080088E029F07F494846BDE8F883089B83B166B941460DB141F08061089A2143381D01F042
S325080089006FFDC146DDF82080D4E74FF08071F0E7DDF82080CEE700F055F9D7F800902A4668
S3250800892021464846FFF744FF18B116B129EA04043C6000F069F9D3E770B170B50C460546C5
S3250800894011F07F4F11D04FF0500383F31188BFF36F8FBFF34F8FFEE74FF0500383F31188F2
S32508008960BFF36F8FBFF34F8FFEE700F02BF92E6826EA04042C6000F047F9304670BD08B5E6
S32508008980FFF7DAFF08BD000008B50A4600230146014802F007FA08BD7F890008EFF3118337
S325080089A04FF0500282F31188BFF36F8FBFF34F8F006883F311887047F8B568B10D46044639
S325080089C011F07F4711D04FF0500383F31188BFF36F8FBFF34F8FFEE74FF0500383F311887A
S325080089E0BFF36F8FBFF34F8FFEE700F10C0601F0F1FA206923682B4323600AE0216832EAD1
S32508008A00010105D111E0216841F0007101F076FD2846B0420ED04568036823F07F4213F0C3
S32508008A20806FEBD121681142F2D013F0807FEAD01743E8E7236823EA0703236001F064FB85
S32508008A402068F8BD08B5FFF7B7FF08BD08B513460A460146014802F0A5F908BD458A00087B
S32508008A6000F1080343604FF0FF328260C360036100230360704700230361704743684B609F
S32508008A809A688A60516099600861036801330360704730B40D68B5F1FF3F11D000F10803F6
S32508008AA01C465B681A68AA42FAD963684B6099608C606160086103680133036030BC704718
S32508008AC00469F2E70369416882688A60416851605A68824206D0002202611A68013A1A60E7
S32508008AE01868704782685A60F5E7000082B0002301930D4B1B68B3F1FF3F08D04FF05003A1
S32508008B0083F31188BFF36F8FBFF34F8FFEE74FF0500383F31188BFF36F8FBFF34F8F019B96
S32508008B20002BFCD002B07047A800002008480068006880F308884FF0000080F3148862B676
S32508008B4061B6BFF34F8FBFF36F8F00DF00BF000008ED00E0DFF80C00016841F470010160EA
S32508008B607047000088ED00E04FF0807340F8043C21F0010140F8081C054B40F80C3C40F8BA
S32508008B80202C6FF0020340F8243C4438704700BFED8A00080000000000000000000000000E
S32508008BA0074B19680868B0E8F04F80F30988BFF36F8F4FF0000080F311887047AFF30080B5
S32508008BC0E08D00204FF0500383F31188BFF36F8FBFF34F8F0B4A136801331360012B00D0A6
S32508008BE070474FF0E023D3F8043D13F0FF0FF7D04FF0500383F31188BFF36F8FBFF34F8FA9
S32508008C00FEE700BFA8000020094B1B6843B94FF0500383F31188BFF36F8FBFF34F8FFEE741
S32508008C20013B034A13600BB983F31188704700BFA800002000000000000000000000000019
S32508008C40EFF30980BFF36F8F154B1A681EF0100F08BF20ED108A20E9F04F10602DE9090097
S32508008C604FF0500080F31188BFF34F8FBFF36F8F01F0ECFA4FF0000080F3118809BC1968A3
S32508008C800868B0E8F04F1EF0100F08BFB0EC108A80F30988BFF36F8F704700BFAFF3008009
S32508008CA0E08D002008B54FF0500383F31188BFF36F8FBFF34F8F01F09BF928B14FF0E023DB
S32508008CC04FF08052C3F8042D002383F3118808BD4FF0E022002313619361054B1B680549A5
S32508008CE0A1FB03139B09013B53610723136170479C000020D34D62104FF0E023D3F8002D43
S32508008D003D4B9A421CD04FF0E023D3F8002D3B4B9A421ED030B583B0394B1A78D2B2019226
S32508008D20FF221A701B78DBB28DF803309DF8033003F05003334A1370334B07221A601BE078
S32508008D404FF0500383F31188BFF36F8FBFF34F8FFEE74FF0500383F31188BFF36F8FBFF33C
S32508008D604F8FFEE7284A1368013B13609DF803305B00DBB28DF803309DF8033013F0800FC4
S32508008D80F0D1214B1B68032B08D04FF0500383F31188BFF36F8FBFF34F8FFEE71B021A4AC8
S32508008DA0136003F4E0631360019BDBB2144A13704FF0E024D4F8203D43F47003C4F8203D4C
S32508008DC0D4F8203D43F07043C4F8203DFFF780FF00250E4B1D60FFF7BDFED4F8343F43F0CA
S32508008DE04043C4F8343FFFF7A1FE01F02FFAFFF77DFE284603B030BD71C20F4170C20F4180
S32508008E0000E400E0780D00207C0D0020A8000020EFF305830F2B0FD9114A9B5CDBB2114AA4
S32508008E2012789A4208D94FF0500383F31188BFF36F8FBFF34F8FFEE74FF0E023D3F80C3DC1
S32508008E4003F4E063084A1268934208D94FF0500383F31188BFF36F8FBFF34F8FFEE77047CB
S32508008E60F0E300E0780D00207C0D0020124A12F0070F1ED0D11D21F00701C1F5004313442A
S32508008E800A460E480260002141601344083B23F007030B48036059601960991A5160136084
S32508008EA0084B1960084B1960084B4FF000421A6070474FF40043E4E7840D0020988D0020C0
S32508008EC0800D00208C8D0020888D0020848D0020164B1A461B688342FBD3516802EB010CAE
S32508008EE0844509D0416800EB010C634509D00360904219D010607047406801445160104667
S32508008F00F0E710B40A4C2468A3420BD05B681944416013681B680360904200D010605DF87D
S32508008F20044B70470460F7E7704700BF988D0020800D002070B5054601F04CF8364B1B68CA
S32508008F40A3B1364B1B681D424ED135B1083515F0070F02D025F007050835002D46D0304B01
S32508008F601B68AB4251D32F4A146804E0FFF77EFFE7E722461C466368AB4202D22368002B29
S32508008F80F7D1254B1B68A34241D0166808362368136063685B1B102B10D9601910F0070F64
S32508008FA008D04FF0500383F31188BFF36F8FBFF34F8FFEE743606560FFF78AFF62681849F3
S32508008FC00B689B1A0B60184909688B4201D216490B60124B1B681343636000232360134AB8
S32508008FE013680133136002E0002600E0002601F08BF816F0070F0CD04FF0500383F3118826
S32508009000BFF36F8FBFF34F8FFEE70026EFE70026EDE7304670BD00BF800D0020848D0020E7
S32508009020888D0020988D00208C8D0020908D0020002834D038B50446A0F1080550F8043CA9
S32508009040174A1268134208D14FF0500383F31188BFF36F8FBFF34F8FFEE750F8081C41B1D5
S325080090604FF0500383F31188BFF36F8FBFF34F8FFEE723EA020340F8043C00F0ABFF54F8AC
S32508009080041C084A13680B4413602846FFF720FF054A13680133136001F036F838BD704754
S325080090A0848D0020888D0020948D00200346406A18B11B6B1868C0F13800704710B504468A
S325080090C0FFF780FDA26BE36B9A4204D00024FFF79BFD204610BD0124F9E710B50446FFF715
S325080090E071FDA36B23B90124FFF78EFD204610BD0024F9E770B504461546866B026C5AB9F1
S3250800910003681BB100200136A66370BD806801F0EFFA0023A360F6E76DB9406801F004FFF6
S32508009120226C636813446360A268934219D3236863602846E7E7C06801F0F6FE226C51422B
S32508009140E3689B1AE3602268934202D2A3680B44E360022D01D00020D5E726B1013E0020DC
S32508009160D1E72846CFE70020CDE70346026C6AB110B50846D9681144D9609C68A14201D3C2
S325080091801968D960D96801F0CFFE10BD704738B50546FFF717FD95F8454064B201E0013CFC
S325080091A064B2002C0ADD6B6A43B105F1240001F05FF90028F3D001F033FAF0E7FF2385F8CD
S325080091C04530FFF721FDFFF7FDFC95F8444064B201E0013C64B2002C0ADD2B6943B105F11D
S325080091E0100001F045F90028F3D001F019FAF0E7FF2385F84430FFF707FD38BD38B5E0B1DC
S325080092000D460446FFF7DEFC2368E26B216C01FB0230A0600020A0636360013A02FB0133EE
S32508009220E360FF2384F8443084F84530FDB9236963B9FFF7E9FC012038BD4FF0500383F383
S325080092401188BFF36F8FBFF34F8FFEE704F1100001F00EF90028ECD04FF0E0234FF080520E
S32508009260C3F8042DBFF34F8FBFF36F8FE1E704F11000FFF7F5FB04F12400FFF7F1FBD8E747
S3250800928038B51D46049C0B4649B92460E063236401212046FFF7B2FF84F84C5038BD226071
S325080092A0F4E740B94FF0500383F31188BFF36F8FBFF34F8FFEE710B584B01C46844653B1DD
S325080092C092B189B94FF0500383F31188BFF36F8FBFF34F8FFEE74FF0500383F31188BFF3E2
S325080092E06F8FBFF34F8FFEE76AB150230393039B502B13D04FF0500383F31188BFF36F8F7C
S32508009300BFF34F8FFEE70029EFD04FF0500383F31188BFF36F8FBFF34F8FFEE7039B01235A
S3250800932084F8463000949DF818306046FFF7A8FF204604B010BD40B94FF0500383F31188F8
S32508009340BFF36F8FBFF34F8FFEE7F0B583B00D461446064601FB00F05030FFF7EBFD074672
S3250800936050B1002380F846300090234600F1500229463046FFF784FF384603B0F0BDF0B5B0
S3250800938085B0019288B10F461D460446B1B1022D20D1E36B012B1DD04FF0500383F3118832
S325080093A0BFF36F8FBFF34F8FFEE74FF0500383F31188BFF36F8FBFF34F8FFEE7036C002B1A
S325080093C0E5D04FF0500383F31188BFF36F8FBFF34F8FFEE701F030F9064658B9019B002BC6
S325080093E048D04FF0500383F31188BFF36F8FBFF34F8FFEE700263DE02A4639462046FFF7F3
S3250800940079FE636A7BB948B14FF0E0234FF08052C3F8042DBFF34F8FBFF36F8FFFF7F4FB69
S32508009420012005B0F0BD04F1240001F021F80028F4D04FF0E0234FF08052C3F8042DBFF39B
S325080094404F8FBFF36F8FE9E7FFF7DEFB0020E8E702A801F097F8012619E0002384F8443085
S3250800946021E0002384F8453023E02046FFF78FFE00F04AFEFFF7A6FBA26BE36B9A42BBD349
S32508009480022DB9D0019B002BDED0002EE0D0FFF7BBFB00F09FFDFFF795FB94F8442052B201
S325080094A0B2F1FF3FD9D094F8452052B2B2F1FF3FD7D0FFF7A9FB01A902A801F06FF8D8B9C0
S325080094C02046FFF7FBFD0028CFD0019904F1100000F06EFF2046FFF75AFE00F015FE002888
S325080094E0C8D14FF0E0234FF08052C3F8042DBFF34F8FBFF36F8FBDE72046FFF748FE00F010
S3250800950003FE00208DE748B108B5002181600160C1600B460A46FFF732FF08BD704710B565
S32508009520024600210120FFF706FF0446FFF7EBFF204610BD10B582B00B46009000221146EA
S325080095400120FFF7AEFE0446FFF7DDFF204602B010BD38B538B10446856801F067F8854215
S325080095600AD0002038BD4FF0500383F31188BFF36F8FBFF34F8FFEE7E368013BE3600BB1A2
S325080095800120EFE71A4619462046FFF7F8FE0120E8E72DE9F84390B10F4616461C460546D5
S325080095A0B1B1022C20D1EB6B012B1DD04FF0500383F31188BFF36F8FBFF34F8FFEE74FF0A8
S325080095C0500383F31188BFF36F8FBFF34F8FFEE7036C002BE5D04FF0500383F31188BFF354
S325080095E06F8FBFF34F8FFEE7FFF712FCEFF311884FF0500383F31188BFF36F8FBFF34F8F8A
S32508009600AA6BEB6B9A4206D3022C04D0002088F31188BDE8F88395F845904FFA89F9AB6B83
S32508009620224639462846FFF765FDB9F1FF3F06D009F101035BB285F845300120E7E76B6AF0
S325080096400BB90120E3E705F1240000F011FF18B126B101203060DAE70120D8E70120D6E763
S32508009660F0B585B0019290B10F460446C1B100F0E3FF064600BB019B002B5ED04FF05003BD
S3250800968083F31188BFF36F8FBFF34F8FFEE74FF0500383F31188BFF36F8FBFF34F8FFEE7C2
S325080096A0036C002BE3D04FF0500383F31188BFF36F8FBFF34F8FFEE700263EE03946204660
S325080096C0FFF753FD013DA563236923B9FFF79CFA012005B0F0BD04F1100000F0C9FE002895
S325080096E0F4D04FF0E0234FF08052C3F8042DBFF34F8FBFF36F8FE9E7FFF786FA0020E8E7E4
S3250800970002A800F03FFF012621E0002384F8443029E0002384F845302BE02046FFF737FD70
S3250800972000F0F2FC09E02046FFF731FD00F0ECFC2046FFF7D2FC00283FD1FFF743FAA56B4D
S32508009740002DBBD1019B002BD6D0002ED8D0FFF75BFA00F03FFCFFF735FA94F844305BB257
S32508009760B3F1FF3FD1D094F845305BB2B3F1FF3FCFD0FFF749FA01A902A800F00FFF002816
S32508009780D1D12046FFF7A9FC0028C6D0019904F1240000F00DFE2046FFF7F9FC00F0B4FCBB
S325080097A00028CAD14FF0E0234FF08052C3F8042DBFF34F8FBFF36F8FBFE7002089E770B5FE
S325080097C084B0019158B10446036C8BB14FF0500383F31188BFF36F8FBFF34F8FFEE74FF0B2
S325080097E0500383F31188BFF36F8FBFF34F8FFEE700F022FF054650B9019B5BB14FF0500335
S3250800980083F31188BFF36F8FBFF34F8FFEE70026354655E0064653E0013BA36323683BB1F8
S3250800982023694BB9FFF7F0F90126304604B070BD01F002F8A060F3E704F1100000F018FE5D
S325080098400028EFD04FF0E0234FF08052C3F8042DBFF34F8FBFF36F8FE4E746B14FF0500340
S3250800986083F31188BFF36F8FBFF34F8FFEE7FFF7CBF9DAE702A800F085FE01252AE00023BB
S3250800988084F8443032E0002384F8453034E0FFF799F9A06800F0E0FE0646FFF7B5F93BE027
S325080098A02046FFF774FC00F02FFC09E02046FFF76EFC00F029FC2046FFF70FFC002842D14D
S325080098C0FFF780F9A36B002BA6D1019B002BC4D0002DCFD0FFF798F900F07CFBFFF772F9E5
S325080098E094F844305BB2B3F1FF3FC8D094F845305BB2B3F1FF3FC6D0FFF786F901A902A884
S3250800990000F04CFE0028D1D12046FFF7E6FB0028C6D02368002BBAD0019904F1240000F057
S3250800992047FD2046FFF733FC00F0EEFB0028C7D14FF0E0234FF08052C3F8042DBFF34F8FE2
S32508009940BFF36F8FBCE70EB900266EE7FFF73AF92046FFF7ABFB0146A06800F011FFFFF7F4
S3250800996053F9F1E780B170B50C460546866800F05DFE864211D021462846FFF720FF80B1C5
S32508009980EB680133EB600CE04FF0500383F31188BFF36F8FBFF34F8FFEE7EB680133EB6063
S325080099A0012070BD2DE9F843B0B10D4690460446D9B1FFF72DFAEFF311874FF0500383F3FD
S325080099C01188BFF36F8FBFF34F8FA66BCEB9002087F31188BDE8F8834FF0500383F3118814
S325080099E0BFF36F8FBFF34F8FFEE7036C002BE0D04FF0500383F31188BFF36F8FBFF34F8F09
S32508009A00FEE794F844904FFA89F929462046FFF7ACFB731EA363B9F1FF3F06D009F1010363
S32508009A205BB284F844300120D2E723690BB90120CEE704F1100000F01BFD30B1B8F1000F75
S32508009A4005D00120C8F80000C2E70120C0E70120BEE700000023072B0CD8074A52F83320E4
S32508009A600AB10133F7E7044A42F8331002EBC30250607047704700BFA08D002070B50446F5
S32508009A800D461646FFF79EF894F844305BB2B3F1FF3F0DD094F845305BB2B3F1FF3F0BD0E6
S32508009AA0FFF7B2F8A36B5BB12046FFF770FB70BD002384F84430EDE7002384F84530EFE719
S32508009AC03246294604F1240000F0B6FCECE70000084B1B681B6823B9074B4FF0FF321A6092
S32508009AE07047044B1B68DB68DB685A68024B1A60704700BFE48D00208C9200202DE9F0472E
S32508009B0080460D4617469946089EDDF824A00A9C9200A521206B01F082F9236B07F1804266
S32508009B20013A03EB820727F00707002D61D04FF0000CBCF10F0F09D815F80C3004EB0C02A5
S32508009B4082F8343013B10CF1010CF2E7002384F84330372E00D93726E662E6640025256584
S32508009B60201DFEF788FF04F11800FEF784FF2461C6F13806A6616462C4F8785184F87C5184
S32508009B804FF49072294604F1580001F048F91B4BE36503F168022266D033636601220023DE
S32508009BA0C4E93C2343F20E33A4F8F8304AF6CD33A4F8FA3041F23423A4F8FC304EF26D63E9
S32508009BC0A4F8FE304DF6EC63A4F800310523A4F802310B23A4F804314A4641463846FEF7CE
S32508009BE0C3FF2060BAF1000F01D0CAF80040BDE8F087002384F83430ABE700BF0C94002058
S32508009C0038B5002407E004EB840293000E481844FEF726FF0134372CF5D90C4D2846FEF748
S32508009C201FFF0B4C2046FEF71BFF0A48FEF718FF0948FEF715FF0948FEF712FF084B1D604D
S32508009C40084B1C6038BD00BFEC8D0020609200207492002098920020C4920020B092002080
S32508009C60E48D0020E88D002010B50446FEF7AAFF224A136801331360214B1B685BB1214B0E
S32508009C801B686BB91E4B1B68DA6AE36A9A4207D81B4B1C6004E01A4B1C601368012B29D090
S32508009CA0194A1368013313606364E06A174B1B68984201D9154B186000EB8000211D144B87
S32508009CC003EB8000FEF7DAFEFEF79EFF0D4B1B687BB10B4B1B68DA6AE36A9A4209D24FF042
S32508009CE0E0234FF08052C3F8042DBFF34F8FBFF36F8F10BDFFF784FFD2E700BF4C9200205A
S32508009D00E08D0020AC920020589200205C920020EC8D002010B50446583001F089F894F804
S32508009D207D3163B1012B11D0022B0ED04FF0500383F31188BFF36F8FBFF34F8FFEE7206BEA
S32508009D40FFF776F92046FFF773F910BD2046FFF76FF9FAE70F4B1B68D3B110B5FEF732FF0A
S32508009D600D4BDB68DC68201DFEF7ACFE0B4A1368013B1360074A1368013B1360FEF744FFE8
S32508009D802046FFF7C7FF034B1B68002BE6D110BD704700BF50920020C49200204C92002027
S32508009DA008B5FFF7D7FF074B1B68012BF9D94FF0E0234FF08052C3F8042DBFF34F8FBFF3B8
S32508009DC06F8FEEE7EC8D002070B504460D46174B1E68174B18680430FEF774FEB4F1FF3FFF
S32508009DE00DD03444124B1B685C60A64210D9114B18680F4B19680431FEF74BFE70BD002D0F
S32508009E00EFD00B4B196804310B48FEF737FEF5E70A4B1868064B19680431FEF73AFE084BB4
S32508009E201B68A342EAD9064B1C60E7E7D8920020E08D0020E88D0020B0920020E48D0020AF
S32508009E408C92002030B587B00B9C8CB10C9DC5B14FF4C0750495049DB5F5C07F1AD04FF0D3
S32508009E60500383F31188BFF36F8FBFF34F8FFEE74FF0500383F31188BFF36F8FBFF34F8F6C
S32508009E80FEE74FF0500383F31188BFF36F8FBFF34F8FFEE7049D0C9D2C63022485F87D41CF
S32508009EA000240394029505AC01940A9C0094FFF725FE0C98FFF7D8FE059807B030BD2DE9E2
S32508009EC0F04385B00746884614461E469000FFF731F808B381464FF4C070FFF72BF805462B
S32508009EE0B0B1C0F83090E5B1002385F87D31039302950D9B01930C9B00933346224641468C
S32508009F003846FFF7FBFD2846FFF7AEFE012005E04846FFF78DF8E6E74FF0FF3005B0BDE813
S32508009F20F0834FF0FF30F9E710B588B000240594069407AA06A905A8FEF722FC059B0293A9
S32508009F40069B019300942346079A1A491A48FFF779FF1A4B186040B100F00EFD012806D025
S32508009F60B0F1FF3F1DD008B010BD0020F6E74FF0500383F31188BFF36F8FBFF34F8F104B49
S32508009F801B6858330F4A13600F4B4FF0FF321A600E4B01221A600E4B00221A60FEF7ACFE0B
S32508009FA0E1E74FF0500383F31188BFF36F8FBFF34F8FFEE798B50008A19D00088892002030
S32508009FC0E08D0020F80000208C920020AC920020D8920020024A136801331360704700BFC4
S32508009FE054920020014B1868704700BFD8920020F8B53A4B1B68002B69D1394B1D68013528
S3250800A0001D60C5B9374B1B681B6843B14FF0500383F31188BFF36F8FBFF34F8FFEE7314A7A
S3250800A0201168314B186810601960304A136801331360FFF74DFD2E4B1B68AB423DD90027B2
S3250800A0402C4B1B68DB6A03EB83039A002A4B9B58012B00D90127294B1B68002B3CD00127BA
S3250800A0603AE001271F4B1B681B6843B31D4B1B68DB68DC6863689D4226D3261D3046FEF767
S3250800A08021FDA36A1BB104F11800FEF71BFDE36A1B4A1268934201D9194A136003EB83037C
S3250800A0A09A00314614481044FEF7E8FCE26A114B1B68DB6A9A42D4D2D4E70027D2E70C4B14
S3250800A0C04FF0FF321A60BBE7094A1360B8E70D4A13680133136000273846F8BD54920020A8
S3250800A0E0D8920020E48D0020E88D0020909200208C920020E08D0020EC8D0020DC9200206E
S3250800A1005C9200209492002038B5354B1B6843B94FF0500383F31188BFF36F8FBFF34F8F10
S3250800A120FEE7FEF74FFD2E4B1A68013A1A601B68002B4FD12B4B1B680BB900244BE000243D
S3250800A140294B1B681BB3284BDB68DC6804F11800FEF7B8FC251D2846FEF7B4FCE06A234B6F
S3250800A1601B68984201D9214B186000EB800029461F4B03EB8000FEF781FCE26A1D4B1B685B
S3250800A180DB6A9A42DCD31C4B01221A60D8E70CB1FFF79EFC194B1C6884B9174B1C68D4B141
S3250800A1A04FF0E0234FF08052C3F8042DBFF34F8FBFF36F8F01240EE0013C07D0FFF718FFDE
S3250800A1C00028F9D00C4B01221A60F5E70B4B00221A60E2E70024FEF717FD204638BD00BFAE
S3250800A1E0549200204C920020989200205C920020EC8D0020E08D0020DC92002094920020FB
S3250800A20010B5A8B10446104B1B6843B14FF0500383F31188BFF36F8FBFF34F8FFEE7FFF73A
S3250800A220D9FE00212046FFF7CFFDFFF76DFF48B94FF0E0234FF08052C3F8042DBFF34F8FBE
S3250800A240BFF36F8F10BD00BF54920020214B1B681BB1214B01221A6070471F4B00221A602D
S3250800A2601E4B1B6803EB83018A001D498A585AB90BB1013BF6E74FF0500383F31188BFF365
S3250800A2806F8FBFF34F8FFEE703EB830082000A4450684068506003EB830C4FEA8C0208326E
S3250800A2A0114488420FD003EB830291000C4A0A445268D1680B4A116008490B60136858336F
S3250800A2C0094A13607047406862469100044A0A445060E8E754920020DC9200205C92002055
S3250800A2E0EC8D0020E08D0020F800002038B50446FEF768FCE4B1251D2846FEF7E3FBA36A5D
S3250800A3001BB104F11800FEF7DDFB29462348FEF7B5FB94F87C31DBB2012B0CD0FEF774FCD7
S3250800A3201F4B1B685BB91F4B1B68A3420ED038BD1C4B1C68DFE7002384F87C31EEE7FEF7A2
S3250800A34041FCFFF7C5FBFEF75FFCECE7144B1B68B3B1154B1B6843B14FF0500383F311881B
S3250800A360BFF36F8FBFF34F8FFEE74FF0E0234FF08052C3F8042DBFF34F8FBFF36F8FD6E76E
S3250800A380064B1A68094B1B689A4203D1054B00221A60CCE7FFF75AFFC9E700BFB092002096
S3250800A3A0AC920020E08D0020549200204C92002058B110B50C46094A11681831FEF769FB12
S3250800A3C001212046FFF700FD10BD4FF0500383F31188BFF36F8FBFF34F8FFEE7E08D0020D4
S3250800A3E070B110B514460246114B1B688BB94FF0500383F31188BFF36F8FBFF34F8FFEE7DE
S3250800A4004FF0500383F31188BFF36F8FBFF34F8FFEE7084B186841F0004181611968183177
S3250800A4201046FEF72BFB01212046FFF7CDFC10BD54920020E08D002038B570B10D4614463B
S3250800A4400A4A11681831FEF719FB0CB14FF0FF3521462846FFF7B8FC38BD4FF0500383F323
S3250800A4601188BFF36F8FBFF34F8FFEE7E08D002038B5C368DC6824B304F118052846FEF7DB
S3250800A48021FB184B1B682BBB251D2846FEF71AFBE06A154B1B68984201D9134B186000EB6A
S3250800A4A080002946114B03EB8000FEF7E7FAE26A0F4B1B68DB6A9A4211D901200D4B1860DA
S3250800A4C038BD4FF0500383F31188BFF36F8FBFF34F8FFEE729460848FEF7D0FAE7E7002047
S3250800A4E0EEE700BF549200205C920020EC8D0020E08D0020DC9200209892002038B51C4B54
S3250800A5001B6843B94FF0500383F31188BFF36F8FBFF34F8FFEE741F000410160C468F4B144
S3250800A520FEF7D0FA251D2846FEF7CCFAE06A114B1B68984201D90F4B186000EB800029465A
S3250800A5400D4B03EB8000FEF799FAE26A0B4B1B68DB6A9A4202D90A4B01221A6038BD4FF058
S3250800A560500383F31188BFF36F8FBFF34F8FFEE7549200205C920020EC8D0020E08D00200C
S3250800A580DC920020034B1B680360034B1B684360704700BF90920020D8920020F8B5C8B10F
S3250800A5A00C460546F9B1FEF70DFB1B4B19686B68C81A2268B2F1FF3F26D0184E36682F68B1
S3250800A5C0B74201D08B4224D9824215D80023236001241AE04FF0500383F31188BFF36F8F12
S3250800A5E0BFF34F8FFEE74FF0500383F31188BFF36F8FBFF34F8FFEE75B1A13442360284655
S3250800A600FFF7C0FF002400E00024FEF7FDFA2046F8BD0124F9E700BFD892002090920020B8
S3250800A620014B01221A607047DC920020014B1868704700BFE08D0020054B1B6833B1054B08
S3250800A6401B680BB1002070470220704701207047AC9200205492002000283ED038B5044654
S3250800A660C36A204A1268D26A93422ED28269002A05DB1C4A1268D26AC2F1380282616169FF
S3250800A68003EB8303184A02EB8303994205D0154B1B68DB6AE362012038BD251D2846FEF78B
S3250800A6A011FA104B1B68D86AE062104B1B68984201D90E4B186000EB800029460A4B03EB9F
S3250800A6C08000FEF7DBF90120E6E7C26C054B1B68DB6A9A4203D30020DEE700207047012060
S3250800A6E0DAE700BFE08D0020EC8D00205C92002000283BD038B504461E4B1B68834208D0A5
S3250800A7004FF0500383F31188BFF36F8FBFF34F8FFEE7036D43B94FF0500383F31188BFF3A6
S3250800A7206F8FBFF34F8FFEE7013B0365C16AC26C91421DD00BB1002038BD051D2846FEF785
S3250800A740C1F9E06CE062C0F13803A3610A4B1B68984201D9084B186000EB80002946074B30
S3250800A76003EB8000FEF78AF90120E5E7002070470020E1E7E08D00205C920020EC8D002005
S3250800A780002846D038B50446036D43B94FF0500383F31188BFF36F8FBFF34F8FFEE7C26CD6
S3250800A7A08A4200D20A46E16A914201D0012B00D038BD184B1B68A34222D0E262A369002B85
S3250800A7C002DBC2F13802A261626901EB8101124B03EB81039A42EBD1251D2846FEF772F9EE
S3250800A7E0E06A0E4B1B68984201D90C4B186000EB80002946084B03EB8000FEF73FF9D7E71C
S3250800A8004FF0500383F31188BFF36F8FBFF34F8FFEE77047E08D0020EC8D00205C92002079
S3250800A820044A136898691368DB6A1268C3F1380393617047E08D0020054B1B6823B1044BE9
S3250800A8401A68136D01331365014B1868704700BFE08D0020064B1A6813682BB901230360B4
S3250800A86023B9D368186870470023F8E700207047E092002008B54160006191420CD8D21AAF
S3250800A88083699A4201D3012008BD011D094B1868FEF7FFF80020F7E79A4201D2994206D2EA
S3250800A8A0011D054B1868FEF7F4F80020ECE70120EAE700BFE4920020E092002030B583B0D7
S3250800A8C0FEF780F9114B1B681BB1FEF79DF903B030BD0F4D2846FEF7C3F80E4C2046FEF7F7
S3250800A8E0BFF80D4B1D600D4B1C60002300930C4B0C4A10210A20FEF7D4FC044B1860002878
S3250800A900E3D00949FFF7A6F8DFE700BF04940020889300209C930020E0920020E4920020A1
S3250800A920B4930020E8920020A0B500082DE9F041079F41B94FF0500383F31188BFF36F8F73
S3250800A940BFF34F8FFEE7064614461D4688468FB1FFF7B4FF3E60C7F81880FD61069B3B6223
S3250800A960381DFEF788F82CB197F8283043F0040387F82830BDE8F08110B588B0FFF79EFF84
S3250800A980124B1B68CBB100240594069407AA06A905A8FDF701FF059B0293069B0193022366
S3250800A9A000932346079A0A490A48FFF74BFA0A4B186010B1012008B010BD4FF0500383F3D0
S3250800A9C01188BFF36F8FBFF34F8FFEE704940020A8B5000869AD0008089400202DE9F0416D
S3250800A9E082B00446884617461D462C20FEF7A2FA064658B1002380F828300190089B009353
S3250800AA002B463A4641462046FFF790FF304602B0BDE8F08110B584B084462C20039003984A
S3250800AA202C2808D04FF0500383F31188BFF36F8FBFF34F8FFEE70398079860B10220079C06
S3250800AA4084F828000194069800906046FFF76EFF079804B010BD4FF0500383F31188BFF305
S3250800AA606F8FBFF34F8FFEE7B8B19C4603461848006858B300B585B000910192029305291D
S3250800AA801CDCFFF7D9FD022810D000231A4669460F480068FEF773FC15E04FF0500383F388
S3250800AAA01188BFF36F8FBFF34F8FFEE70023069A694607480068FEF762FC04E0002362469F
S3250800AAC06946FEF766FD05B05DF804FB002070470494002070B582B01B4B1B681A6862B3F2
S3250800AAE0DB681E68DC68251D2846FDF7EBFF236A2046984794F8283013F0040FECD0A36919
S3250800AB0033449E4207D26360246129460E4B1868FDF7BFFFE0E7002100910B46324620460D
S3250800AB20FFF7A2FF0028D7D14FF0500383F31188BFF36F8FBFF34F8FFEE7044A10680249C9
S3250800AB400860136002B070BDE0920020E492002038B50546FFF746FA0446074B1B688342B3
S3250800AB6005D800232B60044B1C60204638BDFFF7B1FF01232B60F6E7B093002070B582B02A
S3250800AB8006460D4617490968C968CC68201DFDF799FF94F828C01CF0040F08D12CF0010C74
S3250800ABA084F828C0236A2046984702B070BDA16933462A4631442046FFF75CFE0028F1D06B
S3250800ABC0002100910B4632462046FFF74DFF0028E8D14FF0500383F31188BFF36F8FBFF360
S3250800ABE04F8FFEE7E092002070B582B006460C46FFF7F0F901A8FFF7ABFF019B33BB054600
S3250800AC000CB9B04219D224B1124A12681268DAB901242246711B104B1868FEF72FFFFFF7BF
S3250800AC2073FAA8B94FF0E0234FF08052C3F8042DBFF34F8FBFF36F8F0AE0FFF765FA29460B
S3250800AC403046FFF79BFF03E01C46E2E7FFF75CFA02B070BDE49200200494002010B588B05C
S3250800AC6002E0049B002B0FDA002204A93D4B1868FEF7F6FC002873D0049B002BF1DA0799D3
S3250800AC800698059B9847ECE7069C636913B1201DFDF718FF03A8FFF75BFF049B092BE3D8B3
S3250800ACA0DFE803F00505053037500505303794F8283043F0010384F82830059BA1690246B4
S3250800ACC019442046FFF7D6FD0028CDD0236A2046984794F8283013F0040FC5D0A269002188
S3250800ACE000910B46059802442046FFF7BDFE0028BAD14FF0500383F31188BFF36F8FBFF3B4
S3250800AD004F8FFEE794F8283023F0010384F82830AAE794F8283043F0010384F82830059975
S3250800AD20A16131B10346024601442046FFF7A2FD9AE74FF0500383F31188BFF36F8FBFF3CC
S3250800AD404F8FFEE794F8283013F0020F04D023F0010384F8283087E72046FEF769F983E7D6
S3250800AD6008B010BD0494002000B583B001A8FFF771FD0199FFF738FFFFF770FFF6E740B199
S3250800AD8010B50446FDF71EFFE469FDF73DFF204610BD4FF0500383F31188BFF36F8FBFF3D2
S3250800ADA04F8FFEE710B584B014461A466FF0010300930190029103940023694602480068DA
S3250800ADC0FEF7E7FB04B010BD04940020DFF834D0F9F7F4FE0C480D490D4A002302E0D45866
S3250800ADE0C4500433C4188C42F9D30A4A0A4C002301E013600432A242FBD300F06FF8F9F734
S3250800AE007FFCFEE7000001200000002000010020C0B50008000100204C950020FEE7024498
S3250800AE200346934200D1704703F8011BF9E70000294B1B68834270B504464BD0C36943B101
S3250800AE40DB68002B44D1E369196811B1204600F079F8616911B1204600F074F8E16911B1B1
S3250800AE60204600F06FF8216B11B1204600F06AF8616B11B1204600F065F8A16B11B120468C
S3250800AE8000F060F8A16C11B1204600F05BF8616C11B1204600F056F8E16A11B1204600F04E
S3250800AEA051F8236AB3B12046BDE870401847495941B90435E369802DD968F8D1204600F002
S3250800AEC041F8C0E70E68204600F03CF83146EFE70025EFE770BD00BFF800002070B50D4DB9
S3250800AEE00D4C641BA4100026A64209D10B4D0C4C00F080F8641BA4100026A64205D170BD74
S3250800AF0055F8043B98470136EEE755F8043B98470136F2E7B0B50008B0B50008B0B50008EA
S3250800AF20B4B50008704770470A44914200F1FF3300D1704710B511F8014B03F8014F914220
S3250800AF40F9D110BD37B5002944D051F8043C0190002BA1F10404B8BFE41800F03FF81E4A42
S3250800AF600198136833B96360146003B0BDE8304000F03AB8A34208D9256861198B4201BF88
S3250800AF8019685B6849192160EDE71A465B680BB1A342FAD911685518A5420BD12468214477
S3250800AFA05418A3421160E0D11C685B6853600C441460DAE702D90C230360D6E72568611960
S3250800AFC08B4204BF19685B68636004BF491921605460CAE703B030BD489500200148FFF7E5
S3250800AFE0A1BF00BF449500200148FFF79CBF00BF44950020F8B500BFF8BC08BC9E4670475A
S3250800B000F8B500BFF8BC08BC9E46704700000000494E49545F5468726561640010B00008F0
S3250800B02000000000000000000000000000000000000400002F0000000000000000000000CF
S3250800B0404D41494E5F5761746368646F670000004D41494E5F55706461746554696D657245
S3250800B060000000004D41494E5F4576656E745F466C616773000000004D41494E5F43414E9A
S3250800B0805F52785F51756575650000004D41494E5F5468726561640078B000080000000009
S3250800B0A00000000000000000000000000000000064B0000800000000000000000000000066
S3250800B0C08CB0000800000000000000000000000000000000000400002100000000000000F9
S3250800B0E00000000050B0000800000000000000000000000040B00008000000000000000042
S3250800B100000000005045434F5F4576656E745F466C616773000000005045434F5F5570649E
S3250800B12061746554696D6572000000005045434F5F5468726561640004B10008000000002B
S3250800B14000000000000000002CB100080000000000000000000000000000000000040000F8
S3250800B16028000000000000000000000018B100080000000000000000000000005641524897
S3250800B1805F4D7574657800000000000001000000000000000100000001000000000000002C
S3250800B1A0000000C0000040411100000000000000000000000000C842110000000000000014
S3250800B1C0000000000000C8421100000000000000000000000000C842010000000000B84142
S3250800B1E0000020C2000048421100000000002041000000000000404111000000000000C011
S3250800B200000000C0000000000900000000000000000070C20000C842090000000000000012
S3250800B220000070C20000C8420900000000000000000048C200008C420900000000000000DA
S3250800B2400000A0C0000060410900000000000000000020C10000204109000000000000008B
S3250800B260000000000000A0400900000000000000000048C20000164309000000000000006B
S3250800B2800000A0410000F0410900000000000000000000000000A04009000000000000009C
S3250800B2A0000000000000164308000000000000000000000001000000080000000000000016
S3250800B2C000000000FFFFFFFF7CB10008030000000000000000000000414443445F4D75748B
S3250800B2E065780000D8B20008030000000000000000000000414E50495F4D75746578000034
S3250800B300414E50495F4576656E745F466C61677300000000414E50495F546872656164006B
S3250800B320000020410000A040000020410000A04000000000000004419A996D410000044112
S3250800B340F4B2000803000000000000000000000000B3000800000000000000000000000073
S3250800B36014B3000800000000000000000000000000000000000400001000000000000000DC
S3250800B3800000000000040048800000000000000000000000010000000000000000000000D2
S3250800B3A00100000000080048008000000000000000000000010000000000000000000000AD
S3250800B3C0010000000004004808000000000000000000000001000000000000000000000009
S3250800B3E00100000000040048100000000000000000000000010000000000000000000000E1
S3250800B400010000000000004800800000000000000000000001000000000000000000000054
S3250800B42001000000000400484000000001000000000000000100000000000000010000006E
S3250800B44000000000000400482000000001000000000000000100000000000000010000006F
S3250800B46000000000000800480040000001000000000000000100000000000000000000002C
S3250800B480010000000000004800010000010000000000000001000000000000000000000052
S3250800B4A001000000535049445F4576656E745F466C61677300000000535049445F41444349
S3250800B4C05F4D7574657800000404002000000000DCB400080100000002000000B8B40008B5
S3250800B4E0030000000000000000000000A4B4000800000000000000000000000054454D50A5
S3250800B5005F54687265616400FCB400080000000000000000000000000000000000040000AA
S3250800B52018000000000000000000000044656661756C74002CB50008000000000000000037
S3250800B5400000000000000000000200001800000000000000000000000000000000000000C3
S3250800B5600102030406070809A0860100400D0300801A060000350C0040420F0080841E008A
S3250800B58000093D0000127A000024F40000366E010048E801006CDC0249444C450000000075
S3250800B5A0546D725100000000546D722053766300F131000800000000CD310008000000004A
S3250800B5C000FF0000EC010020E401002000000000000000000000000000000000000000004C
S3250800B5E000000000000000000000000000000000000000000000000000000000000000003D
S3250800B6000000000033335340333353400060000000000000E0E90000000000000000000001
S3250800B6200100000000000000010000000100000000000000004000000000000000E80000D1
S3250800B6400000000000000000000000000000000001000000010000000000000000093D0094
S3250800B6600100000010000000AAAAAAAA000000000C94002074940020DC940020000000008B
S3250800B68000000000000000000000000000000000000000000000000000000000000000009C
S3250800B6A0000000000000000000000000000000000000000000000000AC00002000000000B0
S503047682
S7050800ADCD78
